** EXPERIMENTAL (HLL) ** Open Watcom Linker Version 1.6beta1 Limited Availability
Portions Copyright (c) 1985-2002 Sybase, Inc. All Rights Reserved.
Created on:       11/09/01 17:22:47
Executable Image: httpd.dll
creating an OS/2 EMX dynamic link library


                        +------------+
                        |   Groups   |
                        +------------+

Group                           Address              Size
=====                           =======              ====

CGROUP                          0001:00000000        0007df50
DGROUP                          0002:00000000        000047c0



                        +--------------+
                        |   Segments   |
                        +--------------+

Segment                Class          Group          Address         Size
=======                =====          =====          =======         ====

TEXT32                 CODE           CGROUP         0001:00000000   0007df48
________TEXT           CODE           CGROUP         0001:0007df50   00000000
DATA32                 DATA           DGROUP         0002:00000000   000033a0
SET1__os2dll           DATA           DGROUP         0002:000033a0   00000004
SET2__os2dll           DATA           DGROUP         0002:000033a4   00000000
SET3__os2dll           DATA           DGROUP         0002:000033a4   00000004
SET1___CTOR_LIST__     DATA           DGROUP         0002:000033a8   00000004
SET2___CTOR_LIST__     DATA           DGROUP         0002:000033ac   00000000
SET3___CTOR_LIST__     DATA           DGROUP         0002:000033ac   00000004
SET1___DTOR_LIST__     DATA           DGROUP         0002:000033b0   00000004
SET2___DTOR_LIST__     DATA           DGROUP         0002:000033b4   00000000
SET3___DTOR_LIST__     DATA           DGROUP         0002:000033b4   00000004
SET1___crtinit1__      DATA           DGROUP         0002:000033b8   00000004
SET2___crtinit1__      DATA           DGROUP         0002:000033bc   00000000
SET3___crtinit1__      DATA           DGROUP         0002:000033bc   00000004
SET1___crtexit1__      DATA           DGROUP         0002:000033c0   00000004
SET2___crtexit1__      DATA           DGROUP         0002:000033c4   00000000
SET3___crtexit1__      DATA           DGROUP         0002:000033c4   00000004
SET1___eh_frame__      DATA           DGROUP         0002:000033c8   00000004
SET2___eh_frame__      DATA           DGROUP         0002:000033cc   0000002c
SET3___eh_frame__      DATA           DGROUP         0002:000033f8   00000004
SET1___eh_init__       DATA           DGROUP         0002:000033fc   00000004
SET2___eh_init__       DATA           DGROUP         0002:00003400   00000004
SET3___eh_init__       DATA           DGROUP         0002:00003404   00000004
SET1___eh_term__       DATA           DGROUP         0002:00003408   00000004
SET2___eh_term__       DATA           DGROUP         0002:0000340c   00000004
SET3___eh_term__       DATA           DGROUP         0002:00003410   00000004
SET1___fork_parent1__  DATA           DGROUP         0002:00003414   00000004
SET2___fork_parent1__  DATA           DGROUP         0002:00003418   00000000
SET3___fork_parent1__  DATA           DGROUP         0002:00003418   00000004
SET1___fork_child1__   DATA           DGROUP         0002:0000341c   00000004
SET2___fork_child1__   DATA           DGROUP         0002:00003420   00000000
SET3___fork_child1__   DATA           DGROUP         0002:00003420   00000004
________DATA           DATA           DGROUP         0002:00003430   00000000
BSS32                  BSS            DGROUP         0002:00003430   000012b0
c_common               BSS            DGROUP         0002:000046e0   000000e0
________BSS            BSS            DGROUP         0002:000047c0   00000000


                        +----------------+
                        |   Memory Map   |
                        +----------------+

* = unreferenced symbol
+ = symbol only referenced locally

Address        Symbol
=======        ======

Module: U:\usr\lib\dll0.obj({standard input})
0001:00000000* __text
0002:00000000* __data
0002:00000000* ___data_start
0002:00003430* ___bss_start
0002:000033a0+ __os2dll
0002:000033a8  ___CTOR_LIST__
0002:000033b0  ___DTOR_LIST__
0002:000033b8* ___crtinit1__
0002:000033c0* ___crtexit1__
0002:000033c8  ___eh_frame__
0002:000033fc  ___eh_init__
0002:00003408  ___eh_term__
0002:00003414+ ___fork_parent1__
0002:0000341c+ ___fork_child1__
Module: U:\dev\httpd-2.2.20\buildmark.o(buildmark.o)
0001:000000a0  _ap_get_server_built
Module: U:\dev\httpd-2.2.20\server\exports.o(exports.o)
0002:00000050* _ap_hack_apr_allocator_create
0002:00000054* _ap_hack_apr_allocator_destroy
0002:00000058* _ap_hack_apr_allocator_alloc
0002:0000005c* _ap_hack_apr_allocator_free
0002:00000060* _ap_hack_apr_allocator_owner_set
0002:00000064* _ap_hack_apr_allocator_owner_get
0002:00000068* _ap_hack_apr_allocator_max_free_set
0002:0000006c* _ap_hack_apr_allocator_mutex_set
0002:00000070* _ap_hack_apr_allocator_mutex_get
0002:00000074* _ap_hack_apr_atomic_init
0002:00000078* _ap_hack_apr_atomic_read32
0002:0000007c* _ap_hack_apr_atomic_set32
0002:00000080* _ap_hack_apr_atomic_add32
0002:00000084* _ap_hack_apr_atomic_sub32
0002:00000088* _ap_hack_apr_atomic_inc32
0002:0000008c* _ap_hack_apr_atomic_dec32
0002:00000090* _ap_hack_apr_atomic_cas32
0002:00000094* _ap_hack_apr_atomic_xchg32
0002:00000098* _ap_hack_apr_atomic_casptr
0002:0000009c* _ap_hack_apr_atomic_xchgptr
0002:000000a0* _ap_hack_apr_base64_encode_len
0002:000000a4* _ap_hack_apr_base64_encode
0002:000000a8* _ap_hack_apr_base64_encode_binary
0002:000000ac* _ap_hack_apr_base64_decode_len
0002:000000b0* _ap_hack_apr_base64_decode
0002:000000b4* _ap_hack_apr_base64_decode_binary
0002:000000b8* _ap_hack_apr_brigade_create
0002:000000bc* _ap_hack_apr_brigade_destroy
0002:000000c0* _ap_hack_apr_brigade_cleanup
0002:000000c4* _ap_hack_apr_brigade_split_ex
0002:000000c8* _ap_hack_apr_brigade_split
0002:000000cc* _ap_hack_apr_brigade_partition
0002:000000d0* _ap_hack_apr_brigade_length
0002:000000d4* _ap_hack_apr_brigade_flatten
0002:000000d8* _ap_hack_apr_brigade_pflatten
0002:000000dc* _ap_hack_apr_brigade_split_line
0002:000000e0* _ap_hack_apr_brigade_to_iovec
0002:000000e4* _ap_hack_apr_brigade_vputstrs
0002:000000e8* _ap_hack_apr_brigade_write
0002:000000ec* _ap_hack_apr_brigade_writev
0002:000000f0* _ap_hack_apr_brigade_puts
0002:000000f4* _ap_hack_apr_brigade_putc
0002:000000f8* _ap_hack_apr_brigade_putstrs
0002:000000fc* _ap_hack_apr_brigade_printf
0002:00000100* _ap_hack_apr_brigade_vprintf
0002:00000104* _ap_hack_apr_brigade_insert_file
0002:00000108* _ap_hack_apr_bucket_alloc_create
0002:0000010c* _ap_hack_apr_bucket_alloc_create_ex
0002:00000110* _ap_hack_apr_bucket_alloc_destroy
0002:00000114* _ap_hack_apr_bucket_alloc
0002:00000118* _ap_hack_apr_bucket_free
0002:0000011c* _ap_hack_apr_bucket_setaside_noop
0002:00000120* _ap_hack_apr_bucket_setaside_notimpl
0002:00000124* _ap_hack_apr_bucket_split_notimpl
0002:00000128* _ap_hack_apr_bucket_copy_notimpl
0002:0000012c* _ap_hack_apr_bucket_destroy_noop
0002:00000130* _ap_hack_apr_bucket_simple_split
0002:00000134* _ap_hack_apr_bucket_simple_copy
0002:00000138* _ap_hack_apr_bucket_shared_make
0002:0000013c* _ap_hack_apr_bucket_shared_destroy
0002:00000140* _ap_hack_apr_bucket_shared_split
0002:00000144* _ap_hack_apr_bucket_shared_copy
0002:00000148* _ap_hack_apr_bucket_eos_create
0002:0000014c* _ap_hack_apr_bucket_eos_make
0002:00000150* _ap_hack_apr_bucket_flush_create
0002:00000154* _ap_hack_apr_bucket_flush_make
0002:00000158* _ap_hack_apr_bucket_immortal_create
0002:0000015c* _ap_hack_apr_bucket_immortal_make
0002:00000160* _ap_hack_apr_bucket_transient_create
0002:00000164* _ap_hack_apr_bucket_transient_make
0002:00000168* _ap_hack_apr_bucket_heap_create
0002:0000016c* _ap_hack_apr_bucket_heap_make
0002:00000170* _ap_hack_apr_bucket_pool_create
0002:00000174* _ap_hack_apr_bucket_pool_make
0002:00000178* _ap_hack_apr_bucket_socket_create
0002:0000017c* _ap_hack_apr_bucket_socket_make
0002:00000180* _ap_hack_apr_bucket_pipe_create
0002:00000184* _ap_hack_apr_bucket_pipe_make
0002:00000188* _ap_hack_apr_bucket_file_create
0002:0000018c* _ap_hack_apr_bucket_file_make
0002:00000190* _ap_hack_apr_bucket_file_enable_mmap
0002:00000194* _ap_hack_apr_date_checkmask
0002:00000198* _ap_hack_apr_date_parse_http
0002:0000019c* _ap_hack_apr_date_parse_rfc
0002:000001a0* _ap_hack_apr_dbd_init
0002:000001a4* _ap_hack_apr_dbd_get_driver
0002:000001a8* _ap_hack_apr_dbd_open_ex
0002:000001ac* _ap_hack_apr_dbd_open
0002:000001b0* _ap_hack_apr_dbd_close
0002:000001b4* _ap_hack_apr_dbd_name
0002:000001b8* _ap_hack_apr_dbd_native_handle
0002:000001bc* _ap_hack_apr_dbd_check_conn
0002:000001c0* _ap_hack_apr_dbd_set_dbname
0002:000001c4* _ap_hack_apr_dbd_transaction_start
0002:000001c8* _ap_hack_apr_dbd_transaction_end
0002:000001cc* _ap_hack_apr_dbd_transaction_mode_get
0002:000001d0* _ap_hack_apr_dbd_transaction_mode_set
0002:000001d4* _ap_hack_apr_dbd_query
0002:000001d8* _ap_hack_apr_dbd_select
0002:000001dc* _ap_hack_apr_dbd_num_cols
0002:000001e0* _ap_hack_apr_dbd_num_tuples
0002:000001e4* _ap_hack_apr_dbd_get_row
0002:000001e8* _ap_hack_apr_dbd_get_entry
0002:000001ec* _ap_hack_apr_dbd_get_name
0002:000001f0* _ap_hack_apr_dbd_error
0002:000001f4* _ap_hack_apr_dbd_escape
0002:000001f8* _ap_hack_apr_dbd_prepare
0002:000001fc* _ap_hack_apr_dbd_pquery
0002:00000200* _ap_hack_apr_dbd_pselect
0002:00000204* _ap_hack_apr_dbd_pvquery
0002:00000208* _ap_hack_apr_dbd_pvselect
0002:0000020c* _ap_hack_apr_dbd_pbquery
0002:00000210* _ap_hack_apr_dbd_pbselect
0002:00000214* _ap_hack_apr_dbd_pvbquery
0002:00000218* _ap_hack_apr_dbd_pvbselect
0002:0000021c* _ap_hack_apr_dbd_datum_get
0002:00000220* _ap_hack_apr_dbm_open_ex
0002:00000224* _ap_hack_apr_dbm_open
0002:00000228* _ap_hack_apr_dbm_close
0002:0000022c* _ap_hack_apr_dbm_fetch
0002:00000230* _ap_hack_apr_dbm_store
0002:00000234* _ap_hack_apr_dbm_delete
0002:00000238* _ap_hack_apr_dbm_exists
0002:0000023c* _ap_hack_apr_dbm_firstkey
0002:00000240* _ap_hack_apr_dbm_nextkey
0002:00000244* _ap_hack_apr_dbm_freedatum
0002:00000248* _ap_hack_apr_dbm_geterror
0002:0000024c* _ap_hack_apr_dbm_get_usednames_ex
0002:00000250* _ap_hack_apr_dbm_get_usednames
0002:00000254* _ap_hack_apr_dso_load
0002:00000258* _ap_hack_apr_dso_unload
0002:0000025c* _ap_hack_apr_dso_sym
0002:00000260* _ap_hack_apr_dso_error
0002:00000264* _ap_hack_apr_env_get
0002:00000268* _ap_hack_apr_env_set
0002:0000026c* _ap_hack_apr_env_delete
0002:00000270* _ap_hack_apr_strerror
0002:00000274* _ap_hack_apr_stat
0002:00000278* _ap_hack_apr_dir_open
0002:0000027c* _ap_hack_apr_dir_close
0002:00000280* _ap_hack_apr_dir_read
0002:00000284* _ap_hack_apr_dir_rewind
0002:00000288* _ap_hack_apr_filepath_root
0002:0000028c* _ap_hack_apr_filepath_merge
0002:00000290* _ap_hack_apr_filepath_list_split
0002:00000294* _ap_hack_apr_filepath_list_merge
0002:00000298* _ap_hack_apr_filepath_get
0002:0000029c* _ap_hack_apr_filepath_set
0002:000002a0* _ap_hack_apr_filepath_encoding
0002:000002a4* _ap_hack_apr_file_open
0002:000002a8* _ap_hack_apr_file_close
0002:000002ac* _ap_hack_apr_file_remove
0002:000002b0* _ap_hack_apr_file_rename
0002:000002b4* _ap_hack_apr_file_link
0002:000002b8* _ap_hack_apr_file_copy
0002:000002bc* _ap_hack_apr_file_append
0002:000002c0* _ap_hack_apr_file_eof
0002:000002c4* _ap_hack_apr_file_open_stderr
0002:000002c8* _ap_hack_apr_file_open_stdout
0002:000002cc* _ap_hack_apr_file_open_stdin
0002:000002d0* _ap_hack_apr_file_open_flags_stderr
0002:000002d4* _ap_hack_apr_file_open_flags_stdout
0002:000002d8* _ap_hack_apr_file_open_flags_stdin
0002:000002dc* _ap_hack_apr_file_read
0002:000002e0* _ap_hack_apr_file_write
0002:000002e4* _ap_hack_apr_file_writev
0002:000002e8* _ap_hack_apr_file_read_full
0002:000002ec* _ap_hack_apr_file_write_full
0002:000002f0* _ap_hack_apr_file_writev_full
0002:000002f4* _ap_hack_apr_file_putc
0002:000002f8* _ap_hack_apr_file_getc
0002:000002fc* _ap_hack_apr_file_ungetc
0002:00000300* _ap_hack_apr_file_gets
0002:00000304* _ap_hack_apr_file_puts
0002:00000308* _ap_hack_apr_file_flush
0002:0000030c* _ap_hack_apr_file_sync
0002:00000310* _ap_hack_apr_file_datasync
0002:00000314* _ap_hack_apr_file_dup
0002:00000318* _ap_hack_apr_file_dup2
0002:0000031c* _ap_hack_apr_file_setaside
0002:00000320* _ap_hack_apr_file_buffer_set
0002:00000324* _ap_hack_apr_file_buffer_size_get
0002:00000328* _ap_hack_apr_file_seek
0002:0000032c* _ap_hack_apr_file_pipe_create
0002:00000330* _ap_hack_apr_file_pipe_create_ex
0002:00000334* _ap_hack_apr_file_namedpipe_create
0002:00000338* _ap_hack_apr_file_pipe_timeout_get
0002:0000033c* _ap_hack_apr_file_pipe_timeout_set
0002:00000340* _ap_hack_apr_file_lock
0002:00000344* _ap_hack_apr_file_unlock
0002:00000348* _ap_hack_apr_file_name_get
0002:0000034c* _ap_hack_apr_file_data_get
0002:00000350* _ap_hack_apr_file_data_set
0002:00000354* _ap_hack_apr_file_printf
0002:00000358* _ap_hack_apr_file_perms_set
0002:0000035c* _ap_hack_apr_file_attrs_set
0002:00000360* _ap_hack_apr_file_mtime_set
0002:00000364* _ap_hack_apr_dir_make
0002:00000368* _ap_hack_apr_dir_make_recursive
0002:0000036c* _ap_hack_apr_dir_remove
0002:00000370* _ap_hack_apr_file_info_get
0002:00000374* _ap_hack_apr_file_trunc
0002:00000378* _ap_hack_apr_file_flags_get
0002:0000037c* _ap_hack_apr_file_pool_get
0002:00000380* _ap_hack_apr_file_inherit_set
0002:00000384* _ap_hack_apr_file_inherit_unset
0002:00000388* _ap_hack_apr_file_mktemp
0002:0000038c* _ap_hack_apr_temp_dir_get
0002:00000390* _ap_hack_apr_fnmatch
0002:00000394* _ap_hack_apr_fnmatch_test
0002:00000398* _ap_hack_apr_match_glob
0002:0000039c* _ap_hack_apr_initialize
0002:000003a0* _ap_hack_apr_app_initialize
0002:000003a4* _ap_hack_apr_terminate
0002:000003a8* _ap_hack_apr_terminate2
0002:000003ac* _ap_hack_apr_generate_random_bytes
0002:000003b0* _ap_hack_apr_getopt_init
0002:000003b4* _ap_hack_apr_getopt
0002:000003b8* _ap_hack_apr_getopt_long
0002:000003bc* _ap_hack_apr_hashfunc_default
0002:000003c0* _ap_hack_apr_hash_make
0002:000003c4* _ap_hack_apr_hash_make_custom
0002:000003c8* _ap_hack_apr_hash_copy
0002:000003cc* _ap_hack_apr_hash_set
0002:000003d0* _ap_hack_apr_hash_get
0002:000003d4* _ap_hack_apr_hash_first
0002:000003d8* _ap_hack_apr_hash_next
0002:000003dc* _ap_hack_apr_hash_this
0002:000003e0* _ap_hack_apr_hash_count
0002:000003e4* _ap_hack_apr_hash_clear
0002:000003e8* _ap_hack_apr_hash_overlay
0002:000003ec* _ap_hack_apr_hash_merge
0002:000003f0* _ap_hack_apr_hash_do
0002:000003f4* _ap_hack_apr_hash_pool_get
0002:000003f8* _ap_hack_apr_hook_sort_register
0002:000003fc* _ap_hack_apr_hook_sort_all
0002:00000400* _ap_hack_apr_hook_debug_show
0002:00000404* _ap_hack_apr_hook_deregister_all
0002:00000408* _ap_hack_apr_filepath_name_get
0002:0000040c* _ap_hack_apr_vformatter
0002:00000410* _ap_hack_apr_password_get
0002:00000414* _ap_hack_apr_md4_init
0002:00000418* _ap_hack_apr_md4_set_xlate
0002:0000041c* _ap_hack_apr_md4_update
0002:00000420* _ap_hack_apr_md4_final
0002:00000424* _ap_hack_apr_md4
0002:00000428* _ap_hack_apr_md5_init
0002:0000042c* _ap_hack_apr_md5_set_xlate
0002:00000430* _ap_hack_apr_md5_update
0002:00000434* _ap_hack_apr_md5_final
0002:00000438* _ap_hack_apr_md5
0002:0000043c* _ap_hack_apr_md5_encode
0002:00000440* _ap_hack_apr_password_validate
0002:00000444* _ap_hack_apr_memcache_hash
0002:00000448* _ap_hack_apr_memcache_hash_crc32
0002:0000044c* _ap_hack_apr_memcache_hash_default
0002:00000450* _ap_hack_apr_memcache_find_server_hash
0002:00000454* _ap_hack_apr_memcache_find_server_hash_default
0002:00000458* _ap_hack_apr_memcache_add_server
0002:0000045c* _ap_hack_apr_memcache_find_server
0002:00000460* _ap_hack_apr_memcache_enable_server
0002:00000464* _ap_hack_apr_memcache_disable_server
0002:00000468* _ap_hack_apr_memcache_server_create
0002:0000046c* _ap_hack_apr_memcache_create
0002:00000470* _ap_hack_apr_memcache_getp
0002:00000474* _ap_hack_apr_memcache_add_multget_key
0002:00000478* _ap_hack_apr_memcache_multgetp
0002:0000047c* _ap_hack_apr_memcache_set
0002:00000480* _ap_hack_apr_memcache_add
0002:00000484* _ap_hack_apr_memcache_replace
0002:00000488* _ap_hack_apr_memcache_delete
0002:0000048c* _ap_hack_apr_memcache_incr
0002:00000490* _ap_hack_apr_memcache_decr
0002:00000494* _ap_hack_apr_memcache_version
0002:00000498* _ap_hack_apr_memcache_stats
0002:0000049c* _ap_hack_apr_socket_create
0002:000004a0* _ap_hack_apr_socket_shutdown
0002:000004a4* _ap_hack_apr_socket_close
0002:000004a8* _ap_hack_apr_socket_bind
0002:000004ac* _ap_hack_apr_socket_listen
0002:000004b0* _ap_hack_apr_socket_accept
0002:000004b4* _ap_hack_apr_socket_connect
0002:000004b8* _ap_hack_apr_socket_atreadeof
0002:000004bc* _ap_hack_apr_sockaddr_info_get
0002:000004c0* _ap_hack_apr_getnameinfo
0002:000004c4* _ap_hack_apr_parse_addr_port
0002:000004c8* _ap_hack_apr_gethostname
0002:000004cc* _ap_hack_apr_socket_data_get
0002:000004d0* _ap_hack_apr_socket_data_set
0002:000004d4* _ap_hack_apr_socket_send
0002:000004d8* _ap_hack_apr_socket_sendv
0002:000004dc* _ap_hack_apr_socket_sendto
0002:000004e0* _ap_hack_apr_socket_recvfrom
0002:000004e4* _ap_hack_apr_socket_recv
0002:000004e8* _ap_hack_apr_socket_opt_set
0002:000004ec* _ap_hack_apr_socket_timeout_set
0002:000004f0* _ap_hack_apr_socket_opt_get
0002:000004f4* _ap_hack_apr_socket_timeout_get
0002:000004f8* _ap_hack_apr_socket_atmark
0002:000004fc* _ap_hack_apr_socket_addr_get
0002:00000500* _ap_hack_apr_sockaddr_ip_get
0002:00000504* _ap_hack_apr_sockaddr_ip_getbuf
0002:00000508* _ap_hack_apr_sockaddr_equal
0002:0000050c* _ap_hack_apr_socket_type_get
0002:00000510* _ap_hack_apr_getservbyname
0002:00000514* _ap_hack_apr_ipsubnet_create
0002:00000518* _ap_hack_apr_ipsubnet_test
0002:0000051c* _ap_hack_apr_socket_protocol_get
0002:00000520* _ap_hack_apr_socket_pool_get
0002:00000524* _ap_hack_apr_socket_inherit_set
0002:00000528* _ap_hack_apr_socket_inherit_unset
0002:0000052c* _ap_hack_apr_optional_hook_add
0002:00000530* _ap_hack_apr_optional_hook_get
0002:00000534* _ap_hack_apr_dynamic_fn_register
0002:00000538* _ap_hack_apr_dynamic_fn_retrieve
0002:0000053c* _ap_hack_apr_pollset_create
0002:00000540* _ap_hack_apr_pollset_create_ex
0002:00000544* _ap_hack_apr_pollset_destroy
0002:00000548* _ap_hack_apr_pollset_add
0002:0000054c* _ap_hack_apr_pollset_remove
0002:00000550* _ap_hack_apr_pollset_poll
0002:00000554* _ap_hack_apr_poll
0002:00000558* _ap_hack_apr_pollcb_create
0002:0000055c* _ap_hack_apr_pollcb_add
0002:00000560* _ap_hack_apr_pollcb_remove
0002:00000564* _ap_hack_apr_pollcb_poll
0002:00000568* _ap_hack_apr_pool_initialize
0002:0000056c* _ap_hack_apr_pool_terminate
0002:00000570* _ap_hack_apr_pool_create_ex
0002:00000574* _ap_hack_apr_pool_create_core_ex
0002:00000578* _ap_hack_apr_pool_create_unmanaged_ex
0002:0000057c* _ap_hack_apr_pool_create_ex_debug
0002:00000580* _ap_hack_apr_pool_create_core_ex_debug
0002:00000584* _ap_hack_apr_pool_create_unmanaged_ex_debug
0002:00000588* _ap_hack_apr_pool_allocator_get
0002:0000058c* _ap_hack_apr_pool_clear
0002:00000590* _ap_hack_apr_pool_clear_debug
0002:00000594* _ap_hack_apr_pool_destroy
0002:00000598* _ap_hack_apr_pool_destroy_debug
0002:0000059c* _ap_hack_apr_palloc
0002:000005a0* _ap_hack_apr_palloc_debug
0002:000005a4* _ap_hack_apr_pcalloc_debug
0002:000005a8* _ap_hack_apr_pool_abort_set
0002:000005ac* _ap_hack_apr_pool_abort_get
0002:000005b0* _ap_hack_apr_pool_parent_get
0002:000005b4* _ap_hack_apr_pool_is_ancestor
0002:000005b8* _ap_hack_apr_pool_tag
0002:000005bc* _ap_hack_apr_pool_userdata_set
0002:000005c0* _ap_hack_apr_pool_userdata_setn
0002:000005c4* _ap_hack_apr_pool_userdata_get
0002:000005c8* _ap_hack_apr_pool_cleanup_register
0002:000005cc* _ap_hack_apr_pool_pre_cleanup_register
0002:000005d0* _ap_hack_apr_pool_cleanup_kill
0002:000005d4* _ap_hack_apr_pool_child_cleanup_set
0002:000005d8* _ap_hack_apr_pool_cleanup_run
0002:000005dc* _ap_hack_apr_pool_cleanup_null
0002:000005e0* _ap_hack_apr_pool_cleanup_for_exec
0002:000005e4* _ap_hack_apr_os_file_get
0002:000005e8* _ap_hack_apr_os_dir_get
0002:000005ec* _ap_hack_apr_os_sock_get
0002:000005f0* _ap_hack_apr_os_proc_mutex_get
0002:000005f4* _ap_hack_apr_os_exp_time_get
0002:000005f8* _ap_hack_apr_os_imp_time_get
0002:000005fc* _ap_hack_apr_os_shm_get
0002:00000600* _ap_hack_apr_os_thread_get
0002:00000604* _ap_hack_apr_os_threadkey_get
0002:00000608* _ap_hack_apr_os_thread_put
0002:0000060c* _ap_hack_apr_os_threadkey_put
0002:00000610* _ap_hack_apr_os_thread_current
0002:00000614* _ap_hack_apr_os_thread_equal
0002:00000618* _ap_hack_apr_os_file_put
0002:0000061c* _ap_hack_apr_os_pipe_put
0002:00000620* _ap_hack_apr_os_pipe_put_ex
0002:00000624* _ap_hack_apr_os_dir_put
0002:00000628* _ap_hack_apr_os_sock_put
0002:0000062c* _ap_hack_apr_os_sock_make
0002:00000630* _ap_hack_apr_os_proc_mutex_put
0002:00000634* _ap_hack_apr_os_imp_time_put
0002:00000638* _ap_hack_apr_os_exp_time_put
0002:0000063c* _ap_hack_apr_os_shm_put
0002:00000640* _ap_hack_apr_os_dso_handle_put
0002:00000644* _ap_hack_apr_os_dso_handle_get
0002:00000648* _ap_hack_apr_os_uuid_get
0002:0000064c* _ap_hack_apr_os_default_encoding
0002:00000650* _ap_hack_apr_os_locale_encoding
0002:00000654* _ap_hack_apr_proc_mutex_create
0002:00000658* _ap_hack_apr_proc_mutex_child_init
0002:0000065c* _ap_hack_apr_proc_mutex_lock
0002:00000660* _ap_hack_apr_proc_mutex_trylock
0002:00000664* _ap_hack_apr_proc_mutex_unlock
0002:00000668* _ap_hack_apr_proc_mutex_destroy
0002:0000066c* _ap_hack_apr_proc_mutex_cleanup
0002:00000670* _ap_hack_apr_proc_mutex_lockfile
0002:00000674* _ap_hack_apr_proc_mutex_name
0002:00000678* _ap_hack_apr_proc_mutex_defname
0002:0000067c* _ap_hack_apr_proc_mutex_pool_get
0002:00000680* _ap_hack_apr_queue_create
0002:00000684* _ap_hack_apr_queue_push
0002:00000688* _ap_hack_apr_queue_pop
0002:0000068c* _ap_hack_apr_queue_trypush
0002:00000690* _ap_hack_apr_queue_trypop
0002:00000694* _ap_hack_apr_queue_size
0002:00000698* _ap_hack_apr_queue_interrupt_all
0002:0000069c* _ap_hack_apr_queue_term
0002:000006a0* _ap_hack_apr_crypto_sha256_new
0002:000006a4* _ap_hack_apr_random_init
0002:000006a8* _ap_hack_apr_random_standard_new
0002:000006ac* _ap_hack_apr_random_add_entropy
0002:000006b0* _ap_hack_apr_random_insecure_bytes
0002:000006b4* _ap_hack_apr_random_secure_bytes
0002:000006b8* _ap_hack_apr_random_barrier
0002:000006bc* _ap_hack_apr_random_secure_ready
0002:000006c0* _ap_hack_apr_random_insecure_ready
0002:000006c4* _ap_hack_apr_random_after_fork
0002:000006c8* _ap_hack_apr_reslist_create
0002:000006cc* _ap_hack_apr_reslist_destroy
0002:000006d0* _ap_hack_apr_reslist_acquire
0002:000006d4* _ap_hack_apr_reslist_release
0002:000006d8* _ap_hack_apr_reslist_timeout_set
0002:000006dc* _ap_hack_apr_reslist_acquired_count
0002:000006e0* _ap_hack_apr_reslist_invalidate
0002:000006e4* _ap_hack_apr_rmm_init
0002:000006e8* _ap_hack_apr_rmm_destroy
0002:000006ec* _ap_hack_apr_rmm_attach
0002:000006f0* _ap_hack_apr_rmm_detach
0002:000006f4* _ap_hack_apr_rmm_malloc
0002:000006f8* _ap_hack_apr_rmm_realloc
0002:000006fc* _ap_hack_apr_rmm_calloc
0002:00000700* _ap_hack_apr_rmm_free
0002:00000704* _ap_hack_apr_rmm_addr_get
0002:00000708* _ap_hack_apr_rmm_offset_get
0002:0000070c* _ap_hack_apr_rmm_overhead_get
0002:00000710* _ap_hack_apr_sdbm_open
0002:00000714* _ap_hack_apr_sdbm_close
0002:00000718* _ap_hack_apr_sdbm_lock
0002:0000071c* _ap_hack_apr_sdbm_unlock
0002:00000720* _ap_hack_apr_sdbm_fetch
0002:00000724* _ap_hack_apr_sdbm_store
0002:00000728* _ap_hack_apr_sdbm_delete
0002:0000072c* _ap_hack_apr_sdbm_firstkey
0002:00000730* _ap_hack_apr_sdbm_nextkey
0002:00000734* _ap_hack_apr_sdbm_rdonly
0002:00000738* _ap_hack_apr_sha1_base64
0002:0000073c* _ap_hack_apr_sha1_init
0002:00000740* _ap_hack_apr_sha1_update
0002:00000744* _ap_hack_apr_sha1_update_binary
0002:00000748* _ap_hack_apr_sha1_final
0002:0000074c* _ap_hack_apr_shm_create
0002:00000750* _ap_hack_apr_shm_remove
0002:00000754* _ap_hack_apr_shm_destroy
0002:00000758* _ap_hack_apr_shm_attach
0002:0000075c* _ap_hack_apr_shm_detach
0002:00000760* _ap_hack_apr_shm_baseaddr_get
0002:00000764* _ap_hack_apr_shm_size_get
0002:00000768* _ap_hack_apr_shm_pool_get
0002:0000076c* _ap_hack_apr_signal
0002:00000770* _ap_hack_apr_signal_description_get
0002:00000774* _ap_hack_apr_signal_block
0002:00000778* _ap_hack_apr_signal_unblock
0002:0000077c* _ap_hack_apr_strnatcmp
0002:00000780* _ap_hack_apr_strnatcasecmp
0002:00000784* _ap_hack_apr_pstrdup
0002:00000788* _ap_hack_apr_pstrmemdup
0002:0000078c* _ap_hack_apr_pstrndup
0002:00000790* _ap_hack_apr_pmemdup
0002:00000794* _ap_hack_apr_pstrcat
0002:00000798* _ap_hack_apr_pstrcatv
0002:0000079c* _ap_hack_apr_pvsprintf
0002:000007a0* _ap_hack_apr_psprintf
0002:000007a4* _ap_hack_apr_cpystrn
0002:000007a8* _ap_hack_apr_collapse_spaces
0002:000007ac* _ap_hack_apr_tokenize_to_argv
0002:000007b0* _ap_hack_apr_strtok
0002:000007b4* _ap_hack_apr_snprintf
0002:000007b8* _ap_hack_apr_vsnprintf
0002:000007bc* _ap_hack_apr_itoa
0002:000007c0* _ap_hack_apr_ltoa
0002:000007c4* _ap_hack_apr_off_t_toa
0002:000007c8* _ap_hack_apr_strtoff
0002:000007cc* _ap_hack_apr_strtoi64
0002:000007d0* _ap_hack_apr_atoi64
0002:000007d4* _ap_hack_apr_strfsize
0002:000007d8* _ap_hack_apr_strmatch_precompile
0002:000007dc* _ap_hack_apr_table_elts
0002:000007e0* _ap_hack_apr_is_empty_table
0002:000007e4* _ap_hack_apr_is_empty_array
0002:000007e8* _ap_hack_apr_array_make
0002:000007ec* _ap_hack_apr_array_push
0002:000007f0* _ap_hack_apr_array_pop
0002:000007f4* _ap_hack_apr_array_clear
0002:000007f8* _ap_hack_apr_array_cat
0002:000007fc* _ap_hack_apr_array_copy
0002:00000800* _ap_hack_apr_array_copy_hdr
0002:00000804* _ap_hack_apr_array_append
0002:00000808* _ap_hack_apr_array_pstrcat
0002:0000080c* _ap_hack_apr_table_make
0002:00000810* _ap_hack_apr_table_copy
0002:00000814* _ap_hack_apr_table_clone
0002:00000818* _ap_hack_apr_table_clear
0002:0000081c* _ap_hack_apr_table_get
0002:00000820* _ap_hack_apr_table_set
0002:00000824* _ap_hack_apr_table_setn
0002:00000828* _ap_hack_apr_table_unset
0002:0000082c* _ap_hack_apr_table_merge
0002:00000830* _ap_hack_apr_table_mergen
0002:00000834* _ap_hack_apr_table_add
0002:00000838* _ap_hack_apr_table_addn
0002:0000083c* _ap_hack_apr_table_overlay
0002:00000840* _ap_hack_apr_table_do
0002:00000844* _ap_hack_apr_table_vdo
0002:00000848* _ap_hack_apr_table_overlap
0002:0000084c* _ap_hack_apr_table_compress
0002:00000850* _ap_hack_apr_thread_cond_create
0002:00000854* _ap_hack_apr_thread_cond_wait
0002:00000858* _ap_hack_apr_thread_cond_timedwait
0002:0000085c* _ap_hack_apr_thread_cond_signal
0002:00000860* _ap_hack_apr_thread_cond_broadcast
0002:00000864* _ap_hack_apr_thread_cond_destroy
0002:00000868* _ap_hack_apr_thread_cond_pool_get
0002:0000086c* _ap_hack_apr_thread_mutex_create
0002:00000870* _ap_hack_apr_thread_mutex_lock
0002:00000874* _ap_hack_apr_thread_mutex_trylock
0002:00000878* _ap_hack_apr_thread_mutex_unlock
0002:0000087c* _ap_hack_apr_thread_mutex_destroy
0002:00000880* _ap_hack_apr_thread_mutex_pool_get
0002:00000884* _ap_hack_apr_thread_pool_create
0002:00000888* _ap_hack_apr_thread_pool_destroy
0002:0000088c* _ap_hack_apr_thread_pool_push
0002:00000890* _ap_hack_apr_thread_pool_schedule
0002:00000894* _ap_hack_apr_thread_pool_top
0002:00000898* _ap_hack_apr_thread_pool_tasks_cancel
0002:0000089c* _ap_hack_apr_thread_pool_tasks_count
0002:000008a0* _ap_hack_apr_thread_pool_scheduled_tasks_count
0002:000008a4* _ap_hack_apr_thread_pool_threads_count
0002:000008a8* _ap_hack_apr_thread_pool_busy_count
0002:000008ac* _ap_hack_apr_thread_pool_idle_count
0002:000008b0* _ap_hack_apr_thread_pool_idle_max_set
0002:000008b4* _ap_hack_apr_thread_pool_idle_max_get
0002:000008b8* _ap_hack_apr_thread_pool_thread_max_set
0002:000008bc* _ap_hack_apr_thread_pool_thread_max_get
0002:000008c0* _ap_hack_apr_thread_pool_threshold_set
0002:000008c4* _ap_hack_apr_thread_pool_threshold_get
0002:000008c8* _ap_hack_apr_thread_pool_task_owner_get
0002:000008cc* _ap_hack_apr_threadattr_create
0002:000008d0* _ap_hack_apr_threadattr_detach_set
0002:000008d4* _ap_hack_apr_threadattr_detach_get
0002:000008d8* _ap_hack_apr_threadattr_stacksize_set
0002:000008dc* _ap_hack_apr_threadattr_guardsize_set
0002:000008e0* _ap_hack_apr_thread_create
0002:000008e4* _ap_hack_apr_thread_exit
0002:000008e8* _ap_hack_apr_thread_join
0002:000008ec* _ap_hack_apr_thread_yield
0002:000008f0* _ap_hack_apr_thread_once_init
0002:000008f4* _ap_hack_apr_thread_once
0002:000008f8* _ap_hack_apr_thread_detach
0002:000008fc* _ap_hack_apr_thread_data_get
0002:00000900* _ap_hack_apr_thread_data_set
0002:00000904* _ap_hack_apr_threadkey_private_create
0002:00000908* _ap_hack_apr_threadkey_private_get
0002:0000090c* _ap_hack_apr_threadkey_private_set
0002:00000910* _ap_hack_apr_threadkey_private_delete
0002:00000914* _ap_hack_apr_threadkey_data_get
0002:00000918* _ap_hack_apr_threadkey_data_set
0002:0000091c* _ap_hack_apr_procattr_create
0002:00000920* _ap_hack_apr_procattr_io_set
0002:00000924* _ap_hack_apr_procattr_child_in_set
0002:00000928* _ap_hack_apr_procattr_child_out_set
0002:0000092c* _ap_hack_apr_procattr_child_err_set
0002:00000930* _ap_hack_apr_procattr_dir_set
0002:00000934* _ap_hack_apr_procattr_cmdtype_set
0002:00000938* _ap_hack_apr_procattr_detach_set
0002:0000093c* _ap_hack_apr_procattr_limit_set
0002:00000940* _ap_hack_apr_procattr_child_errfn_set
0002:00000944* _ap_hack_apr_procattr_error_check_set
0002:00000948* _ap_hack_apr_procattr_addrspace_set
0002:0000094c* _ap_hack_apr_procattr_user_set
0002:00000950* _ap_hack_apr_procattr_group_set
0002:00000954* _ap_hack_apr_proc_fork
0002:00000958* _ap_hack_apr_proc_create
0002:0000095c* _ap_hack_apr_proc_wait
0002:00000960* _ap_hack_apr_proc_wait_all_procs
0002:00000964* _ap_hack_apr_proc_detach
0002:00000968* _ap_hack_apr_proc_other_child_register
0002:0000096c* _ap_hack_apr_proc_other_child_unregister
0002:00000970* _ap_hack_apr_proc_other_child_alert
0002:00000974* _ap_hack_apr_proc_other_child_refresh
0002:00000978* _ap_hack_apr_proc_other_child_refresh_all
0002:0000097c* _ap_hack_apr_proc_kill
0002:00000980* _ap_hack_apr_pool_note_subprocess
0002:00000984* _ap_hack_apr_thread_pool_get
0002:00000988* _ap_hack_apr_thread_rwlock_create
0002:0000098c* _ap_hack_apr_thread_rwlock_rdlock
0002:00000990* _ap_hack_apr_thread_rwlock_tryrdlock
0002:00000994* _ap_hack_apr_thread_rwlock_wrlock
0002:00000998* _ap_hack_apr_thread_rwlock_trywrlock
0002:0000099c* _ap_hack_apr_thread_rwlock_unlock
0002:000009a0* _ap_hack_apr_thread_rwlock_destroy
0002:000009a4* _ap_hack_apr_thread_rwlock_pool_get
0002:000009a8* _ap_hack_apr_time_now
0002:000009ac* _ap_hack_apr_time_ansi_put
0002:000009b0* _ap_hack_apr_time_exp_tz
0002:000009b4* _ap_hack_apr_time_exp_gmt
0002:000009b8* _ap_hack_apr_time_exp_lt
0002:000009bc* _ap_hack_apr_time_exp_get
0002:000009c0* _ap_hack_apr_time_exp_gmt_get
0002:000009c4* _ap_hack_apr_sleep
0002:000009c8* _ap_hack_apr_rfc822_date
0002:000009cc* _ap_hack_apr_ctime
0002:000009d0* _ap_hack_apr_strftime
0002:000009d4* _ap_hack_apr_time_clock_hires
0002:000009d8* _ap_hack_apr_uri_port_of_scheme
0002:000009dc* _ap_hack_apr_uri_unparse
0002:000009e0* _ap_hack_apr_uri_parse
0002:000009e4* _ap_hack_apr_uri_parse_hostinfo
0002:000009e8* _ap_hack_apr_uid_current
0002:000009ec* _ap_hack_apr_uid_name_get
0002:000009f0* _ap_hack_apr_uid_get
0002:000009f4* _ap_hack_apr_uid_homepath_get
0002:000009f8* _ap_hack_apr_gid_name_get
0002:000009fc* _ap_hack_apr_gid_get
0002:00000a00* _ap_hack_apr_uuid_get
0002:00000a04* _ap_hack_apr_uuid_format
0002:00000a08* _ap_hack_apr_uuid_parse
0002:00000a0c* _ap_hack_apr_version
0002:00000a10* _ap_hack_apr_version_string
0002:00000a14* _ap_hack_apr_xlate_open
0002:00000a18* _ap_hack_apr_xlate_sb_get
0002:00000a1c* _ap_hack_apr_xlate_conv_buffer
0002:00000a20* _ap_hack_apr_xlate_conv_byte
0002:00000a24* _ap_hack_apr_xlate_close
0002:00000a28* _ap_hack_apr_text_append
0002:00000a2c* _ap_hack_apr_xml_parser_create
0002:00000a30* _ap_hack_apr_xml_parse_file
0002:00000a34* _ap_hack_apr_xml_parser_feed
0002:00000a38* _ap_hack_apr_xml_parser_done
0002:00000a3c* _ap_hack_apr_xml_parser_geterror
0002:00000a40* _ap_hack_apr_xml_to_text
0002:00000a44* _ap_hack_apr_xml_empty_elem
0002:00000a48* _ap_hack_apr_xml_quote_string
0002:00000a4c* _ap_hack_apr_xml_quote_elem
0002:00000a50* _ap_hack_apr_xml_insert_uri
0002:00000a54* _ap_hack_apu_version
0002:00000a58* _ap_hack_apu_version_string
0002:00000a5c* _ap_hack_ap_listen_pre_config
0002:00000a60* _ap_hack_ap_setup_listeners
0002:00000a64* _ap_hack_ap_close_listeners
0002:00000a68* _ap_hack_ap_set_listenbacklog
0002:00000a6c* _ap_hack_ap_set_listener
0002:00000a70* _ap_hack_ap_set_send_buffer_size
0002:00000a74* _ap_hack_ap_set_receive_buffer_size
0002:00000a78* _ap_hack_ap_mpm_run
0002:00000a7c* _ap_hack_ap_graceful_stop_signalled
0002:00000a80* _ap_hack_ap_os_create_privileged_process
0002:00000a84* _ap_hack_ap_mpm_query
0002:00000a88* _ap_hack_ap_register_provider
0002:00000a8c* _ap_hack_ap_lookup_provider
0002:00000a90* _ap_hack_ap_list_provider_names
0002:00000a94* _ap_hack_ap_regcomp
0002:00000a98* _ap_hack_ap_regexec
0002:00000a9c* _ap_hack_ap_regerror
0002:00000aa0* _ap_hack_ap_regfree
0002:00000aa4* _ap_hack_ap_get_module_config
0002:00000aa8* _ap_hack_ap_set_module_config
0002:00000aac* _ap_hack_ap_set_string_slot
0002:00000ab0* _ap_hack_ap_set_int_slot
0002:00000ab4* _ap_hack_ap_method_is_limited
0002:00000ab8* _ap_hack_ap_set_string_slot_lower
0002:00000abc* _ap_hack_ap_set_flag_slot
0002:00000ac0* _ap_hack_ap_set_file_slot
0002:00000ac4* _ap_hack_ap_set_deprecated
0002:00000ac8* _ap_hack_ap_server_root_relative
0002:00000acc* _ap_hack_ap_add_module
0002:00000ad0* _ap_hack_ap_remove_module
0002:00000ad4* _ap_hack_ap_add_loaded_module
0002:00000ad8* _ap_hack_ap_remove_loaded_module
0002:00000adc* _ap_hack_ap_find_module_name
0002:00000ae0* _ap_hack_ap_find_linked_module
0002:00000ae4* _ap_hack_ap_pcfg_openfile
0002:00000ae8* _ap_hack_ap_pcfg_open_custom
0002:00000aec* _ap_hack_ap_cfg_getline
0002:00000af0* _ap_hack_ap_cfg_getc
0002:00000af4* _ap_hack_ap_cfg_closefile
0002:00000af8* _ap_hack_ap_soak_end_container
0002:00000afc* _ap_hack_ap_build_cont_config
0002:00000b00* _ap_hack_ap_build_config
0002:00000b04* _ap_hack_ap_walk_config
0002:00000b08* _ap_hack_ap_check_cmd_context
0002:00000b0c* _ap_hack_ap_single_module_configure
0002:00000b10* _ap_hack_ap_setup_prelinked_modules
0002:00000b14* _ap_hack_ap_show_directives
0002:00000b18* _ap_hack_ap_show_modules
0002:00000b1c* _ap_hack_ap_show_mpm
0002:00000b20* _ap_hack_ap_read_config
0002:00000b24* _ap_hack_ap_run_rewrite_args
0002:00000b28* _ap_hack_ap_register_hooks
0002:00000b2c* _ap_hack_ap_fixup_virtual_hosts
0002:00000b30* _ap_hack_ap_create_request_config
0002:00000b34* _ap_hack_ap_create_per_dir_config
0002:00000b38* _ap_hack_ap_merge_per_dir_configs
0002:00000b3c* _ap_hack_ap_create_conn_config
0002:00000b40* _ap_hack_ap_parse_htaccess
0002:00000b44* _ap_hack_ap_init_virtual_host
0002:00000b48* _ap_hack_ap_process_resource_config
0002:00000b4c* _ap_hack_ap_process_config_tree
0002:00000b50* _ap_hack_ap_invoke_handler
0002:00000b54* _ap_hack_ap_find_command
0002:00000b58* _ap_hack_ap_find_command_in_modules
0002:00000b5c* _ap_hack_ap_set_config_vectors
0002:00000b60* _ap_hack_ap_hook_header_parser
0002:00000b64* _ap_hack_ap_hook_get_header_parser
0002:00000b68* _ap_hack_ap_run_header_parser
0002:00000b6c* _ap_hack_ap_hook_pre_config
0002:00000b70* _ap_hack_ap_hook_get_pre_config
0002:00000b74* _ap_hack_ap_run_pre_config
0002:00000b78* _ap_hack_ap_hook_test_config
0002:00000b7c* _ap_hack_ap_hook_get_test_config
0002:00000b80* _ap_hack_ap_run_test_config
0002:00000b84* _ap_hack_ap_hook_post_config
0002:00000b88* _ap_hack_ap_hook_get_post_config
0002:00000b8c* _ap_hack_ap_run_post_config
0002:00000b90* _ap_hack_ap_hook_open_logs
0002:00000b94* _ap_hack_ap_hook_get_open_logs
0002:00000b98* _ap_hack_ap_run_open_logs
0002:00000b9c* _ap_hack_ap_hook_child_init
0002:00000ba0* _ap_hack_ap_hook_get_child_init
0002:00000ba4* _ap_hack_ap_run_child_init
0002:00000ba8* _ap_hack_ap_hook_handler
0002:00000bac* _ap_hack_ap_hook_get_handler
0002:00000bb0* _ap_hack_ap_run_handler
0002:00000bb4* _ap_hack_ap_hook_quick_handler
0002:00000bb8* _ap_hack_ap_hook_get_quick_handler
0002:00000bbc* _ap_hack_ap_run_quick_handler
0002:00000bc0* _ap_hack_ap_hook_optional_fn_retrieve
0002:00000bc4* _ap_hack_ap_hook_get_optional_fn_retrieve
0002:00000bc8* _ap_hack_ap_run_optional_fn_retrieve
0002:00000bcc* _ap_hack_ap_process_connection
0002:00000bd0* _ap_hack_ap_flush_conn
0002:00000bd4* _ap_hack_ap_lingering_close
0002:00000bd8* _ap_hack_ap_hook_create_connection
0002:00000bdc* _ap_hack_ap_hook_get_create_connection
0002:00000be0* _ap_hack_ap_run_create_connection
0002:00000be4* _ap_hack_ap_hook_pre_connection
0002:00000be8* _ap_hack_ap_hook_get_pre_connection
0002:00000bec* _ap_hack_ap_run_pre_connection
0002:00000bf0* _ap_hack_ap_hook_process_connection
0002:00000bf4* _ap_hack_ap_hook_get_process_connection
0002:00000bf8* _ap_hack_ap_run_process_connection
0002:00000bfc* _ap_hack_ap_bucket_eoc_make
0002:00000c00* _ap_hack_ap_bucket_eoc_create
0002:00000c04* _ap_hack_ap_allow_options
0002:00000c08* _ap_hack_ap_allow_overrides
0002:00000c0c* _ap_hack_ap_default_type
0002:00000c10* _ap_hack_ap_document_root
0002:00000c14* _ap_hack_ap_get_remote_host
0002:00000c18* _ap_hack_ap_get_remote_logname
0002:00000c1c* _ap_hack_ap_construct_url
0002:00000c20* _ap_hack_ap_get_server_name
0002:00000c24* _ap_hack_ap_get_server_port
0002:00000c28* _ap_hack_ap_get_limit_req_body
0002:00000c2c* _ap_hack_ap_get_limit_xml_body
0002:00000c30* _ap_hack_ap_custom_response
0002:00000c34* _ap_hack_ap_is_recursion_limit_exceeded
0002:00000c38* _ap_hack_ap_exists_config_define
0002:00000c3c* _ap_hack_ap_core_translate
0002:00000c40* _ap_hack_ap_auth_type
0002:00000c44* _ap_hack_ap_auth_name
0002:00000c48* _ap_hack_ap_satisfies
0002:00000c4c* _ap_hack_ap_requires
0002:00000c50* _ap_hack_ap_register_request_note
0002:00000c54* _ap_hack_ap_get_request_note
0002:00000c58* _ap_hack_ap_add_per_dir_conf
0002:00000c5c* _ap_hack_ap_add_per_url_conf
0002:00000c60* _ap_hack_ap_add_file_conf
0002:00000c64* _ap_hack_ap_limit_section
0002:00000c68* _ap_hack_ap_get_server_protocol
0002:00000c6c* _ap_hack_ap_set_server_protocol
0002:00000c70* _ap_hack_ap_hook_get_mgmt_items
0002:00000c74* _ap_hack_ap_hook_get_get_mgmt_items
0002:00000c78* _ap_hack_ap_run_get_mgmt_items
0002:00000c7c* _ap_hack_ap_open_stderr_log
0002:00000c80* _ap_hack_ap_replace_stderr_log
0002:00000c84* _ap_hack_ap_log_error
0002:00000c88* _ap_hack_ap_log_perror
0002:00000c8c* _ap_hack_ap_log_rerror
0002:00000c90* _ap_hack_ap_log_cerror
0002:00000c94* _ap_hack_ap_error_log2stderr
0002:00000c98* _ap_hack_ap_log_pid
0002:00000c9c* _ap_hack_ap_read_pid
0002:00000ca0* _ap_hack_ap_open_piped_log
0002:00000ca4* _ap_hack_ap_open_piped_log_ex
0002:00000ca8* _ap_hack_ap_close_piped_log
0002:00000cac* _ap_hack_ap_hook_error_log
0002:00000cb0* _ap_hack_ap_hook_get_error_log
0002:00000cb4* _ap_hack_ap_run_error_log
0002:00000cb8* _ap_hack_ap_hook_insert_error_filter
0002:00000cbc* _ap_hack_ap_hook_get_insert_error_filter
0002:00000cc0* _ap_hack_ap_run_insert_error_filter
0002:00000cc4* _ap_hack_ap_get_mime_headers
0002:00000cc8* _ap_hack_ap_get_mime_headers_core
0002:00000ccc* _ap_hack_ap_finalize_request_protocol
0002:00000cd0* _ap_hack_ap_send_error_response
0002:00000cd4* _ap_hack_ap_set_content_length
0002:00000cd8* _ap_hack_ap_set_keepalive
0002:00000cdc* _ap_hack_ap_rationalize_mtime
0002:00000ce0* _ap_hack_ap_make_content_type
0002:00000ce4* _ap_hack_ap_setup_make_content_type
0002:00000ce8* _ap_hack_ap_make_etag
0002:00000cec* _ap_hack_ap_set_etag
0002:00000cf0* _ap_hack_ap_set_last_modified
0002:00000cf4* _ap_hack_ap_meets_conditions
0002:00000cf8* _ap_hack_ap_send_fd
0002:00000cfc* _ap_hack_ap_method_register
0002:00000d00* _ap_hack_ap_method_registry_init
0002:00000d04* _ap_hack_ap_make_method_list
0002:00000d08* _ap_hack_ap_copy_method_list
0002:00000d0c* _ap_hack_ap_method_in_list
0002:00000d10* _ap_hack_ap_method_list_add
0002:00000d14* _ap_hack_ap_method_list_remove
0002:00000d18* _ap_hack_ap_clear_method_list
0002:00000d1c* _ap_hack_ap_set_content_type
0002:00000d20* _ap_hack_ap_rputc
0002:00000d24* _ap_hack_ap_rputs
0002:00000d28* _ap_hack_ap_rwrite
0002:00000d2c* _ap_hack_ap_rvputs
0002:00000d30* _ap_hack_ap_vrprintf
0002:00000d34* _ap_hack_ap_rprintf
0002:00000d38* _ap_hack_ap_rflush
0002:00000d3c* _ap_hack_ap_index_of_response
0002:00000d40* _ap_hack_ap_get_status_line
0002:00000d44* _ap_hack_ap_setup_client_block
0002:00000d48* _ap_hack_ap_should_client_block
0002:00000d4c* _ap_hack_ap_get_client_block
0002:00000d50* _ap_hack_ap_discard_request_body
0002:00000d54* _ap_hack_ap_note_auth_failure
0002:00000d58* _ap_hack_ap_note_basic_auth_failure
0002:00000d5c* _ap_hack_ap_note_digest_auth_failure
0002:00000d60* _ap_hack_ap_get_basic_auth_pw
0002:00000d64* _ap_hack_ap_parse_uri
0002:00000d68* _ap_hack_ap_getline
0002:00000d6c* _ap_hack_ap_rgetline_core
0002:00000d70* _ap_hack_ap_method_number_of
0002:00000d74* _ap_hack_ap_method_name_of
0002:00000d78* _ap_hack_ap_hook_post_read_request
0002:00000d7c* _ap_hack_ap_hook_get_post_read_request
0002:00000d80* _ap_hack_ap_run_post_read_request
0002:00000d84* _ap_hack_ap_hook_log_transaction
0002:00000d88* _ap_hack_ap_hook_get_log_transaction
0002:00000d8c* _ap_hack_ap_run_log_transaction
0002:00000d90* _ap_hack_ap_hook_http_scheme
0002:00000d94* _ap_hack_ap_hook_get_http_scheme
0002:00000d98* _ap_hack_ap_run_http_scheme
0002:00000d9c* _ap_hack_ap_hook_default_port
0002:00000da0* _ap_hack_ap_hook_get_default_port
0002:00000da4* _ap_hack_ap_run_default_port
0002:00000da8* _ap_hack_ap_bucket_error_make
0002:00000dac* _ap_hack_ap_bucket_error_create
0002:00000db0* _ap_hack_ap_byterange_filter
0002:00000db4* _ap_hack_ap_http_header_filter
0002:00000db8* _ap_hack_ap_content_length_filter
0002:00000dbc* _ap_hack_ap_old_write_filter
0002:00000dc0* _ap_hack_ap_set_sub_req_protocol
0002:00000dc4* _ap_hack_ap_finalize_sub_req_protocol
0002:00000dc8* _ap_hack_ap_send_interim_response
0002:00000dcc* _ap_hack_ap_process_request_internal
0002:00000dd0* _ap_hack_ap_sub_req_lookup_uri
0002:00000dd4* _ap_hack_ap_sub_req_lookup_file
0002:00000dd8* _ap_hack_ap_sub_req_lookup_dirent
0002:00000ddc* _ap_hack_ap_sub_req_method_uri
0002:00000de0* _ap_hack_ap_sub_req_output_filter
0002:00000de4* _ap_hack_ap_run_sub_req
0002:00000de8* _ap_hack_ap_destroy_sub_req
0002:00000dec* _ap_hack_ap_internal_redirect
0002:00000df0* _ap_hack_ap_internal_redirect_handler
0002:00000df4* _ap_hack_ap_internal_fast_redirect
0002:00000df8* _ap_hack_ap_some_auth_required
0002:00000dfc* _ap_hack_ap_is_initial_req
0002:00000e00* _ap_hack_ap_update_mtime
0002:00000e04* _ap_hack_ap_allow_methods
0002:00000e08* _ap_hack_ap_allow_standard_methods
0002:00000e0c* _ap_hack_ap_die
0002:00000e10* _ap_hack_ap_hook_create_request
0002:00000e14* _ap_hack_ap_hook_get_create_request
0002:00000e18* _ap_hack_ap_run_create_request
0002:00000e1c* _ap_hack_ap_hook_translate_name
0002:00000e20* _ap_hack_ap_hook_get_translate_name
0002:00000e24* _ap_hack_ap_run_translate_name
0002:00000e28* _ap_hack_ap_hook_map_to_storage
0002:00000e2c* _ap_hack_ap_hook_get_map_to_storage
0002:00000e30* _ap_hack_ap_run_map_to_storage
0002:00000e34* _ap_hack_ap_hook_check_user_id
0002:00000e38* _ap_hack_ap_hook_get_check_user_id
0002:00000e3c* _ap_hack_ap_run_check_user_id
0002:00000e40* _ap_hack_ap_hook_fixups
0002:00000e44* _ap_hack_ap_hook_get_fixups
0002:00000e48* _ap_hack_ap_run_fixups
0002:00000e4c* _ap_hack_ap_hook_type_checker
0002:00000e50* _ap_hack_ap_hook_get_type_checker
0002:00000e54* _ap_hack_ap_run_type_checker
0002:00000e58* _ap_hack_ap_hook_access_checker
0002:00000e5c* _ap_hack_ap_hook_get_access_checker
0002:00000e60* _ap_hack_ap_run_access_checker
0002:00000e64* _ap_hack_ap_hook_auth_checker
0002:00000e68* _ap_hack_ap_hook_get_auth_checker
0002:00000e6c* _ap_hack_ap_run_auth_checker
0002:00000e70* _ap_hack_ap_hook_insert_filter
0002:00000e74* _ap_hack_ap_hook_get_insert_filter
0002:00000e78* _ap_hack_ap_run_insert_filter
0002:00000e7c* _ap_hack_ap_location_walk
0002:00000e80* _ap_hack_ap_directory_walk
0002:00000e84* _ap_hack_ap_file_walk
0002:00000e88* _ap_hack_ap_init_vhost_config
0002:00000e8c* _ap_hack_ap_fini_vhost_config
0002:00000e90* _ap_hack_ap_vhost_iterate_given_conn
0002:00000e94* _ap_hack_ap_update_vhost_given_ip
0002:00000e98* _ap_hack_ap_update_vhost_from_headers
0002:00000e9c* _ap_hack_ap_matches_request_vhost
0002:00000ea0* _ap_hack_ap_get_server_revision
0002:00000ea4* _ap_hack_ap_get_server_version
0002:00000ea8* _ap_hack_ap_get_server_banner
0002:00000eac* _ap_hack_ap_get_server_description
0002:00000eb0* _ap_hack_ap_add_version_component
0002:00000eb4* _ap_hack_ap_get_server_built
0002:00000eb8* _ap_hack_ap_field_noparam
0002:00000ebc* _ap_hack_ap_ht_time
0002:00000ec0* _ap_hack_ap_getword
0002:00000ec4* _ap_hack_ap_getword_nc
0002:00000ec8* _ap_hack_ap_getword_white
0002:00000ecc* _ap_hack_ap_getword_white_nc
0002:00000ed0* _ap_hack_ap_getword_nulls
0002:00000ed4* _ap_hack_ap_getword_nulls_nc
0002:00000ed8* _ap_hack_ap_getword_conf
0002:00000edc* _ap_hack_ap_getword_conf_nc
0002:00000ee0* _ap_hack_ap_resolve_env
0002:00000ee4* _ap_hack_ap_size_list_item
0002:00000ee8* _ap_hack_ap_get_list_item
0002:00000eec* _ap_hack_ap_find_list_item
0002:00000ef0* _ap_hack_ap_get_token
0002:00000ef4* _ap_hack_ap_find_token
0002:00000ef8* _ap_hack_ap_find_last_token
0002:00000efc* _ap_hack_ap_is_url
0002:00000f00* _ap_hack_ap_unescape_url
0002:00000f04* _ap_hack_ap_unescape_url_keep2f
0002:00000f08* _ap_hack_ap_unescape_url_keep2f_ex
0002:00000f0c* _ap_hack_ap_no2slash
0002:00000f10* _ap_hack_ap_getparents
0002:00000f14* _ap_hack_ap_escape_path_segment
0002:00000f18* _ap_hack_ap_os_escape_path
0002:00000f1c* _ap_hack_ap_escape_html
0002:00000f20* _ap_hack_ap_escape_html2
0002:00000f24* _ap_hack_ap_escape_logitem
0002:00000f28* _ap_hack_ap_escape_errorlog_item
0002:00000f2c* _ap_hack_ap_construct_server
0002:00000f30* _ap_hack_ap_escape_shell_cmd
0002:00000f34* _ap_hack_ap_count_dirs
0002:00000f38* _ap_hack_ap_make_dirstr_prefix
0002:00000f3c* _ap_hack_ap_make_dirstr_parent
0002:00000f40* _ap_hack_ap_make_full_path
0002:00000f44* _ap_hack_ap_os_is_path_absolute
0002:00000f48* _ap_hack_ap_is_matchexp
0002:00000f4c* _ap_hack_ap_strcmp_match
0002:00000f50* _ap_hack_ap_strcasecmp_match
0002:00000f54* _ap_hack_ap_strcasestr
0002:00000f58* _ap_hack_ap_stripprefix
0002:00000f5c* _ap_hack_ap_pbase64decode
0002:00000f60* _ap_hack_ap_pbase64encode
0002:00000f64* _ap_hack_ap_pregcomp
0002:00000f68* _ap_hack_ap_pregfree
0002:00000f6c* _ap_hack_ap_pregsub
0002:00000f70* _ap_hack_ap_content_type_tolower
0002:00000f74* _ap_hack_ap_str_tolower
0002:00000f78* _ap_hack_ap_ind
0002:00000f7c* _ap_hack_ap_rind
0002:00000f80* _ap_hack_ap_escape_quotes
0002:00000f84* _ap_hack_ap_append_pid
0002:00000f88* _ap_hack_ap_timeout_parameter_parse
0002:00000f8c* _ap_hack_ap_is_rdirectory
0002:00000f90* _ap_hack_ap_is_directory
0002:00000f94* _ap_hack_ap_log_assert
0002:00000f98* _ap_hack_ap_psignature
0002:00000f9c* _ap_hack_ap_strchr
0002:00000fa0* _ap_hack_ap_strchr_c
0002:00000fa4* _ap_hack_ap_strrchr
0002:00000fa8* _ap_hack_ap_strrchr_c
0002:00000fac* _ap_hack_ap_strstr
0002:00000fb0* _ap_hack_ap_strstr_c
0002:00000fb4* _ap_hack_ap_uname2id
0002:00000fb8* _ap_hack_ap_gname2id
0002:00000fbc* _ap_hack_ap_hook_monitor
0002:00000fc0* _ap_hack_ap_hook_get_monitor
0002:00000fc4* _ap_hack_ap_run_monitor
0002:00000fc8* _ap_hack_ap_exists_scoreboard_image
0002:00000fcc* _ap_hack_ap_increment_counts
0002:00000fd0* _ap_hack_ap_calc_scoreboard_size
0002:00000fd4* _ap_hack_ap_create_sb_handle
0002:00000fd8* _ap_hack_ap_update_child_status
0002:00000fdc* _ap_hack_ap_update_child_status_from_indexes
0002:00000fe0* _ap_hack_ap_get_scoreboard_worker
0002:00000fe4* _ap_hack_ap_get_scoreboard_process
0002:00000fe8* _ap_hack_ap_get_scoreboard_global
0002:00000fec* _ap_hack_ap_get_scoreboard_lb
0002:00000ff0* _ap_hack_ap_hook_pre_mpm
0002:00000ff4* _ap_hack_ap_hook_get_pre_mpm
0002:00000ff8* _ap_hack_ap_run_pre_mpm
0002:00000ffc* _ap_hack_ap_get_brigade
0002:00001000* _ap_hack_ap_pass_brigade
0002:00001004* _ap_hack_ap_register_input_filter
0002:00001008* _ap_hack_ap_register_output_filter
0002:0000100c* _ap_hack_ap_register_output_filter_protocol
0002:00001010* _ap_hack_ap_add_input_filter
0002:00001014* _ap_hack_ap_add_input_filter_handle
0002:00001018* _ap_hack_ap_get_input_filter_handle
0002:0000101c* _ap_hack_ap_add_output_filter
0002:00001020* _ap_hack_ap_add_output_filter_handle
0002:00001024* _ap_hack_ap_get_output_filter_handle
0002:00001028* _ap_hack_ap_remove_input_filter
0002:0000102c* _ap_hack_ap_remove_output_filter
0002:00001030* _ap_hack_ap_save_brigade
0002:00001034* _ap_hack_ap_filter_flush
0002:00001038* _ap_hack_ap_fflush
0002:0000103c* _ap_hack_ap_fputstrs
0002:00001040* _ap_hack_ap_fprintf
0002:00001044* _ap_hack_ap_filter_protocol
0002:00001048* _ap_hack_ap_md5
0002:0000104c* _ap_hack_ap_md5_binary
0002:00001050* _ap_hack_ap_md5contextTo64
0002:00001054* _ap_hack_ap_md5digest
0002:00001058* _ap_hack_ap_create_environment
0002:0000105c* _ap_hack_ap_find_path_info
0002:00001060* _ap_hack_ap_add_cgi_vars
0002:00001064* _ap_hack_ap_add_common_vars
0002:00001068* _ap_hack_ap_scan_script_header_err
0002:0000106c* _ap_hack_ap_scan_script_header_err_brigade
0002:00001070* _ap_hack_ap_scan_script_header_err_strs
0002:00001074* _ap_hack_ap_scan_script_header_err_core
0002:00001078* _ap_hack_ap_explode_recent_localtime
0002:0000107c* _ap_hack_ap_explode_recent_gmt
0002:00001080* _ap_hack_ap_recent_ctime
0002:00001084* _ap_hack_ap_recent_rfc822_date
0002:00001088* _ap_hack_ap_xml_parse_input
0002:0000108c* _ap_hack_ap_basic_http_header
0002:00001090* _ap_hack_ap_send_http_trace
0002:00001094* _ap_hack_ap_send_http_options
0002:00003430  _ap_ugly_hack
Module: U:\dev\httpd-2.2.20\modules.o(modules.o)
0002:000010a0  _ap_prelinked_modules
0002:000010c0  _ap_prelinked_module_symbols
0002:000010f0  _ap_preloaded_modules
Module: U:\dev\httpd-2.2.20\server\.libs\main.lib(main.o)
0001:00000fac  _main
0001:00001e9c* _suck_in_APR
0001:00000fac* main
Module: U:\usr\lib\tcpipv4\libc_dll.lib(swapl.obj)
0001:00001eb0  __swapl
Module: U:\extras\lib\apr-1.lib(apr_pools.o)
0001:0000241c  _apr_allocator_create
0001:00002464  _apr_allocator_destroy
0001:000024a0  _apr_allocator_mutex_set
0001:000024b0  _apr_allocator_mutex_get
0001:000024bc  _apr_allocator_owner_set
0001:000024cc  _apr_allocator_owner_get
0001:000024d8  _apr_allocator_max_free_set
0001:00002530  _apr_allocator_alloc
0001:00002738  _apr_allocator_free
0001:00002824  _apr_palloc
0001:00002bb0* _apr_pcalloc
0001:00002be4  _apr_pool_destroy
0001:00002ddc  _apr_pool_clear
0001:00002f74  _apr_pool_terminate
0001:00002fb4  _apr_pool_create_ex
0001:000032ec  _apr_pool_initialize
0001:000033c4  _apr_pool_create_unmanaged_ex
0001:000036b0  _apr_pool_create_core_ex
0001:000036bc  _apr_pvsprintf
0001:00003908  _apr_psprintf
0001:0000392c  _apr_pool_abort_set
0001:0000393c  _apr_pool_abort_get
0001:00003948  _apr_pool_parent_get
0001:00003954  _apr_pool_allocator_get
0001:00003960  _apr_pool_is_ancestor
0001:0000398c  _apr_pool_tag
0001:0000399c  _apr_pool_userdata_get
0001:000039e4  _apr_pool_cleanup_register
0001:00003a34  _apr_pool_userdata_setn
0001:00003a9c  _apr_pool_userdata_set
0001:00003b50  _apr_pool_pre_cleanup_register
0001:00003b98  _apr_pool_cleanup_kill
0001:00003c0c  _apr_pool_child_cleanup_set
0001:00003c44  _apr_pool_cleanup_run
0001:00003c74  _apr_pool_cleanup_for_exec
0001:00003c7c  _apr_pool_cleanup_null
0001:00003c84  _apr_pool_note_subprocess
0001:00003cb8  _apr_palloc_debug
0001:00003cc4  _apr_pcalloc_debug
0001:00003cd0  _apr_pool_clear_debug
0001:00003cdc  _apr_pool_destroy_debug
0001:00003ce8  _apr_pool_create_ex_debug
0001:00003cf4  _apr_pool_create_core_ex_debug
0001:00003d00  _apr_pool_create_unmanaged_ex_debug
Module: U:\extras\lib\apr-1.lib(ia32.o)
0001:00003d10  _apr_atomic_init
0001:00003d18  _apr_atomic_read32
0001:00003d24  _apr_atomic_set32
0001:00003d34  _apr_atomic_add32
0001:00003d44  _apr_atomic_sub32
0001:00003d54  _apr_atomic_inc32
0001:00003d68  _apr_atomic_dec32
0001:00003d7c  _apr_atomic_cas32
0001:00003d90  _apr_atomic_xchg32
0001:00003da0  _apr_atomic_casptr
0001:00003db4  _apr_atomic_xchgptr
Module: U:\extras\lib\aprutil-1.lib(apr_base64.o)
0001:00003dd0  _apr_base64_decode_len
0001:00003e04  _apr_base64_decode_binary
0001:00003f68  _apr_base64_decode
0001:00003f8c  _apr_base64_encode_len
0001:00003fac  _apr_base64_encode_binary
0001:000040d8  _apr_base64_encode
Module: U:\extras\lib\aprutil-1.lib(apr_brigade.o)
0001:00004240  _apr_brigade_cleanup
0001:0000429c  _apr_brigade_destroy
0001:000042cc  _apr_brigade_create
0001:00004320  _apr_brigade_split_ex
0001:00004398  _apr_brigade_split
0001:000043bc  _apr_brigade_partition
0001:00004584  _apr_brigade_length
0001:00004630  _apr_brigade_flatten
0001:000046c4  _apr_brigade_pflatten
0001:00004724  _apr_brigade_to_iovec
0001:000047b0  _apr_brigade_write
0001:0000496c  _apr_brigade_putc
0001:000049a4  _apr_brigade_vputstrs
0001:00004a04  _apr_brigade_split_line
0001:00004bb8  _apr_brigade_writev
0001:00004e60  _apr_brigade_puts
0001:00004eec  _apr_brigade_putstrs
0001:00004f14  _apr_brigade_vprintf
0001:00004fa4  _apr_brigade_printf
0001:00004fd4  _apr_brigade_insert_file
Module: U:\extras\lib\aprutil-1.lib(apr_buckets_alloc.o)
0001:00005180  _apr_bucket_alloc_create_ex
0001:000051cc  _apr_bucket_alloc_create
0001:00005210  _apr_bucket_alloc_destroy
0001:0000524c  _apr_bucket_alloc
0001:000052e8  _apr_bucket_free
Module: U:\extras\lib\aprutil-1.lib(apr_buckets.o)
0001:00005320  _apr_bucket_setaside_noop
0001:00005328  _apr_bucket_setaside_notimpl
0001:00005334  _apr_bucket_split_notimpl
0001:00005340  _apr_bucket_copy_notimpl
0001:0000534c  _apr_bucket_destroy_noop
Module: U:\extras\lib\aprutil-1.lib(apr_buckets_simple.o)
0001:000053b4  _apr_bucket_simple_copy
0001:000053ec  _apr_bucket_simple_split
0001:00005448  _apr_bucket_immortal_make
0001:00005550  _apr_bucket_type_immortal
0001:00005474  _apr_bucket_immortal_create
0001:000054c4  _apr_bucket_transient_make
0001:00005580  _apr_bucket_type_transient
0001:000054f0  _apr_bucket_transient_create
Module: U:\extras\lib\aprutil-1.lib(apr_buckets_refcount.o)
0001:000055a0  _apr_bucket_shared_split
0001:000055c8  _apr_bucket_shared_copy
0001:000055f0  _apr_bucket_shared_destroy
0001:00005608  _apr_bucket_shared_make
Module: U:\extras\lib\aprutil-1.lib(apr_buckets_eos.o)
0001:0000564c  _apr_bucket_eos_make
0001:000056d0  _apr_bucket_type_eos
0001:00005678  _apr_bucket_eos_create
Module: U:\extras\lib\aprutil-1.lib(apr_buckets_flush.o)
0001:0000570c  _apr_bucket_flush_make
0001:00005790  _apr_bucket_type_flush
0001:00005738  _apr_bucket_flush_create
Module: U:\extras\lib\aprutil-1.lib(apr_buckets_heap.o)
0001:00005804  _apr_bucket_heap_make
0001:00005910  _apr_bucket_type_heap
0001:000058b8  _apr_bucket_heap_create
Module: U:\extras\lib\aprutil-1.lib(apr_buckets_pool.o)
0001:00005a00  _apr_bucket_pool_make
0001:00005b00  _apr_bucket_type_pool
0001:00005a9c  _apr_bucket_pool_create
Module: U:\extras\lib\aprutil-1.lib(apr_buckets_socket.o)
0001:00005b20  _apr_bucket_socket_make
0001:00005d50  _apr_bucket_type_socket
0001:00005b4c  _apr_bucket_socket_create
Module: U:\extras\lib\aprutil-1.lib(apr_buckets_pipe.o)
0001:00005d70  _apr_bucket_pipe_make
0001:00005fc0  _apr_bucket_type_pipe
0001:00005d9c  _apr_bucket_pipe_create
Module: U:\extras\lib\aprutil-1.lib(apr_buckets_file.o)
0001:00006360  _apr_bucket_type_file
0001:0000627c  _apr_bucket_file_make
0001:000062d8  _apr_bucket_file_create
0001:00006344  _apr_bucket_file_enable_mmap
Module: U:\extras\lib\aprutil-1.lib(apr_date.o)
0001:00006380  _apr_date_checkmask
0001:000064bc  _apr_date_parse_http
0001:000068ec  _apr_date_parse_rfc
Module: U:\extras\lib\aprutil-1.lib(apr_dbd.o)
0001:00007194* _apr_dbd_mutex_lock
0001:000071ac* _apr_dbd_mutex_unlock
0001:000071c4  _apr_dbd_init
0001:000072b0  _apr_dbd_get_driver
0001:00007410  _apr_dbd_open_ex
0001:0000749c  _apr_dbd_open
0001:000074cc  _apr_dbd_transaction_start
0001:00007520  _apr_dbd_transaction_end
0001:00007554  _apr_dbd_transaction_mode_get
0001:0000756c  _apr_dbd_transaction_mode_set
0001:00007588  _apr_dbd_close
0001:000075a0  _apr_dbd_name
0001:000075ac  _apr_dbd_native_handle
0001:000075c4  _apr_dbd_check_conn
0001:000075e0  _apr_dbd_set_dbname
0001:00007604  _apr_dbd_query
0001:00007628  _apr_dbd_select
0001:00007660  _apr_dbd_num_cols
0001:00007678  _apr_dbd_num_tuples
0001:00007690  _apr_dbd_get_row
0001:000076b8  _apr_dbd_get_entry
0001:000076d4  _apr_dbd_get_name
0001:000076f0  _apr_dbd_error
0001:0000770c  _apr_dbd_escape
0001:00007730  _apr_dbd_prepare
0001:00007bdc  _apr_dbd_pquery
0001:00007c14  _apr_dbd_pselect
0001:00007c50  _apr_dbd_pvquery
0001:00007c80  _apr_dbd_pvselect
0001:00007cb8  _apr_dbd_pbquery
0001:00007cf0  _apr_dbd_pbselect
0001:00007d2c  _apr_dbd_pvbquery
0001:00007d5c  _apr_dbd_pvbselect
0001:00007d94  _apr_dbd_datum_get
Module: U:\extras\lib\aprutil-1.lib(apr_dbm.o)
0001:000080f8  _apr_dbm_open_ex
0001:00008148  _apr_dbm_open
0001:00008180  _apr_dbm_close
0001:00008194  _apr_dbm_fetch
0001:000081ac  _apr_dbm_store
0001:000081c4  _apr_dbm_delete
0001:000081d8  _apr_dbm_exists
0001:000081ec  _apr_dbm_firstkey
0001:00008200  _apr_dbm_nextkey
0001:00008214  _apr_dbm_freedatum
0001:00008228  _apr_dbm_geterror
0001:00008270  _apr_dbm_get_usednames_ex
0001:000082b8  _apr_dbm_get_usednames
0001:000082e8* _apr_posix_perms2mode
Module: U:\extras\lib\apr-1.lib(dso.o)
0001:00008354  _apr_dso_load
0001:00008444  _apr_dso_unload
0001:0000846c  _apr_dso_sym
0001:00008518  _apr_dso_error
0001:000085a8  _apr_os_dso_handle_put
0001:000085e8  _apr_os_dso_handle_get
Module: U:\extras\lib\apr-1.lib(env.o)
0001:00008600  _apr_env_get
0001:00008628  _apr_env_set
0001:00008650  _apr_env_delete
Module: U:\extras\lib\apr-1.lib(errorcodes.o)
0001:00008f70  _apr_strerror
Module: U:\extras\lib\apr-1.lib(filestat.o)
0001:000093a0  _apr_file_info_get_locked
0001:00009554  _apr_file_info_get
0001:00009760  _apr_file_perms_set
0001:0000976c  _apr_stat
0001:00009958  _apr_file_attrs_set
0001:00009a28  _apr_file_mtime_set
Module: U:\extras\lib\apr-1.lib(dir.o)
0001:00009ad0  _apr_dir_open
0001:00009b70  _apr_dir_close
0001:00009bc0  _apr_dir_read
0001:00009d48  _apr_dir_rewind
0001:00009d54  _apr_dir_make
0001:00009d98  _apr_dir_remove
0001:00009dcc  _apr_os_dir_get
0001:00009dec  _apr_os_dir_put
Module: U:\extras\lib\apr-1.lib(filepath.o)
0001:00009e40  _apr_filepath_root
0001:0000a1d0  _apr_filepath_merge
0001:0000af9c  _apr_filepath_list_split
0001:0000afc8  _apr_filepath_list_merge
0001:0000aff4  _apr_filepath_encoding
Module: U:\extras\lib\apr-1.lib(filesys.o)
0001:0000b010  _filepath_root_test
0001:0000b048  _filepath_drive_get
0001:0000b0fc  _filepath_root_case
0001:0000b15c  _apr_filepath_get
0001:0000b1fc  _apr_filepath_set
0001:0000b250  _c_is_fnchar
Module: U:\extras\lib\apr-1.lib(open.o)
0001:0000b3c8  _apr_unix_file_cleanup
0001:0000b3fc  _apr_unix_child_file_cleanup
0001:0000b40c  _apr_file_open
0001:0000b79c  _apr_file_cleanup
0001:0000b71c  _apr_file_close
0001:0000b7a8  _apr_file_remove
0001:0000b7c8  _apr_file_rename
0001:0000b82c  _apr_os_file_get
0001:0000b840  _apr_os_file_put
0001:0000b8ec  _apr_file_eof
0001:0000b90c  _apr_file_open_flags_stderr
0001:0000b940  _apr_file_open_flags_stdout
0001:0000b974  _apr_file_open_flags_stdin
0001:0000b9a8  _apr_file_open_stderr
0001:0000b9cc  _apr_file_open_stdout
0001:0000b9f0  _apr_file_open_stdin
0001:0000ba14  _apr_file_pool_get
0001:0000ba20  _apr_file_inherit_set
0001:0000ba74  _apr_file_inherit_unset
0001:0000baa0  _apr_file_link
Module: U:\extras\lib\apr-1.lib(copy.o)
0001:0000bc78  _apr_file_copy
0001:0000bc9c  _apr_file_append
Module: U:\extras\lib\apr-1.lib(readwrite.o)
0001:0000bd0c  _apr_file_putc
0001:0000bd5c  _apr_file_ungetc
0001:0000bd8c  _apr_file_puts
0001:0000bdc8  _apr_file_flush_locked
0001:0000be34  _apr_file_writev
0001:0000bf18  _apr_file_flush
0001:0000bf80  _apr_file_write
0001:0000c1cc  _apr_file_read
0001:0000c4a4  _apr_file_getc
0001:0000c4cc  _apr_file_sync
0001:0000c4d8  _apr_file_datasync
0001:0000c4e4  _apr_file_gets
0001:0000c584  _apr_file_printf
0001:0000c604* _apr_file_check_read
Module: U:\extras\lib\apr-1.lib(fullrw.o)
0001:0000c650  _apr_file_read_full
0001:0000c6a0  _apr_file_write_full
0001:0000c6f0  _apr_file_writev_full
Module: U:\extras\lib\apr-1.lib(filedup.o)
0001:0000c958  _apr_file_dup
0001:0000c994  _apr_file_dup2
0001:0000c9ac  _apr_file_setaside
Module: U:\extras\lib\apr-1.lib(buffer.o)
0001:0000cae0  _apr_file_buffer_set
0001:0000cb6c  _apr_file_buffer_size_get
Module: U:\extras\lib\apr-1.lib(seek.o)
0001:0000cc1c  _apr_file_seek
0001:0000cd3c  _apr_file_trunc
Module: U:\extras\lib\apr-1.lib(pipe.o)
0001:0000cd9c  _apr_file_pipe_create
0001:0000d0e4  _apr_file_namedpipe_create
0001:0000d0f0  _apr_file_pipe_timeout_set
0001:0000d16c  _apr_file_pipe_create_ex
0001:0000d210  _apr_file_pipe_timeout_get
0001:0000d238  _apr_os_pipe_put_ex
0001:0000d2b8  _apr_os_pipe_put
Module: U:\extras\lib\apr-1.lib(flock.o)
0001:0000d2f0  _apr_file_lock
0001:0000d350  _apr_file_unlock
Module: U:\extras\lib\apr-1.lib(fileacc.o)
0001:0000d3a0  _apr_file_name_get
0001:0000d3b4  _apr_file_flags_get
0001:0000d3c0* _apr_unix_perms2mode
0001:0000d434  _apr_unix_mode2perms
0001:0000d4a8  _apr_file_data_get
0001:0000d4bc  _apr_file_data_set
Module: U:\extras\lib\apr-1.lib(dir_make_recurse.o)
0001:0000d4f0  _apr_dir_make_recursive
Module: U:\extras\lib\apr-1.lib(mktemp.o)
0001:0000d630  _apr_file_mktemp
Module: U:\extras\lib\apr-1.lib(tempdir.o)
0001:0000d7bc  _apr_temp_dir_get
Module: U:\extras\lib\apr-1.lib(apr_fnmatch.o)
0001:0000d920  _apr_fnmatch
0001:0000e338  _apr_fnmatch_test
0001:0000e388  _apr_match_glob
Module: U:\extras\lib\apr-1.lib(start.o)
0001:0000e4c0  _apr_initialize
0001:0000e544  _apr_app_initialize
0001:0000e550  _apr_terminate
0001:0000e570  _apr_terminate2
Module: U:\extras\lib\apr-1.lib(rand.o)
0001:0000e580  _apr_os_uuid_get
0001:0000e5a8* _randbyte
0001:0000e5d4  _apr_generate_random_bytes
Module: U:\extras\lib\apr-1.lib(getopt.o)
0001:0000e69c  _apr_getopt_init
0001:0000e780  _apr_getopt
0001:0000e9d4  _apr_getopt_long
Module: U:\extras\lib\apr-1.lib(apr_hash.o)
0001:0000edc0  _apr_hashfunc_default
0001:0000ef30  _apr_hash_make
0001:0000ef84  _apr_hash_make_custom
0001:0000efa0  _apr_hash_next
0001:0000eff0  _apr_hash_first
0001:0000f068  _apr_hash_this
0001:0000f0a4  _apr_hash_copy
0001:0000f170  _apr_hash_get
0001:0000f19c  _apr_hash_set
0001:0000f288  _apr_hash_count
0001:0000f294  _apr_hash_clear
0001:0000f31c  _apr_hash_merge
0001:0000f568  _apr_hash_overlay
0001:0000f59c  _apr_hash_do
0001:0000f654  _apr_hash_pool_get
Module: U:\extras\lib\aprutil-1.lib(apr_hooks.o)
0001:0000f674  _apr_hook_sort_register
0001:0000f708  _apr_hook_sort_all
0001:0000fc4c  _apr_hook_deregister_all
0001:0000fcb0  _apr_hook_debug_show
0001:0000fddc  _apr_optional_hook_get
0001:0000fe28  _apr_optional_hook_add
0001:0000ff44  _apr_dynamic_fn_retrieve
0001:0000ff8c  _apr_dynamic_fn_register
0002:000034e0  _apr_hook_global_pool
0002:000034e4  _apr_hook_debug_enabled
0002:000034e8  _apr_hook_debug_current
0002:000034ec* _apr_global_hook_pool
0002:000034f0* _apr_debug_module_hooks
0002:000034f4* _apr_current_hooking_module
Module: U:\extras\lib\apr-1.lib(apr_cpystrn.o)
0001:0000fff0  _apr_cpystrn
0001:00010028  _apr_tokenize_to_argv
0001:00010298  _apr_filepath_name_get
0001:000102c8  _apr_collapse_spaces
Module: U:\extras\lib\apr-1.lib(apr_snprintf.o)
0001:000107ac  _apr_vformatter
0001:000122c4  _apr_snprintf
0001:00012344  _apr_vsnprintf
Module: U:\extras\lib\apr-1.lib(apr_getpass.o)
0001:00012460  _apr_password_get
Module: U:\extras\lib\aprutil-1.lib(apr_md4.o)
0001:00012a24  _apr_md4_init
0001:00012a60  _apr_md4_set_xlate
0001:00012a9c  _apr_md4_update
0001:00012c60  _apr_md4_final
0001:00012cf4  _apr_md4
Module: U:\extras\lib\aprutil-1.lib(apr_md5.o)
0001:000136ec  _apr_md5_init
0001:00013728  _apr_md5_set_xlate
0001:00013764  _apr_md5_update
0001:00013780  _apr_md5_final
0001:00013814  _apr_md5
0001:00013888  _apr_md5_encode
0001:00013e6c  _apr_password_validate
Module: U:\extras\lib\aprutil-1.lib(apr_memcache.o)
0001:00014404  _apr_memcache_add_server
0001:00014448  _apr_memcache_find_server_hash_default
0001:000145e4  _apr_memcache_find_server_hash
0001:00014624  _apr_memcache_find_server
0001:0001467c  _apr_memcache_enable_server
0001:00014694  _apr_memcache_disable_server
0001:000147ac  _apr_memcache_server_create
0001:00014894  _apr_memcache_create
0001:00014908  _apr_memcache_hash_crc32
0001:00014944  _apr_memcache_hash_default
0001:00014988  _apr_memcache_hash
0001:00014dac  _apr_memcache_set
0001:00014df4  _apr_memcache_add
0001:00014e40  _apr_memcache_replace
0001:00014e94  _apr_memcache_getp
0001:00015190  _apr_memcache_delete
0001:00015348  _apr_memcache_incr
0001:00015374  _apr_memcache_decr
0001:000153a0  _apr_memcache_version
0001:000154c0  _apr_memcache_add_multget_key
0001:00015550  _apr_memcache_multgetp
0001:00015f90  _apr_memcache_stats
Module: U:\extras\lib\apr-1.lib(sockets.o)
0001:00016a58  _apr_socket_protocol_get
0001:00016a6c  _apr_socket_create
0001:00016b5c  _apr_socket_shutdown
0001:00016b98  _apr_socket_close
0001:00016bc8  _apr_socket_bind
0001:00016c34  _apr_socket_listen
0001:00016c70  _apr_socket_accept
0001:00016d98  _apr_socket_connect
0001:00016e20  _apr_socket_type_get
0001:00016e34  _apr_socket_data_get
0001:00016e80  _apr_socket_data_set
0001:00016eec  _apr_os_sock_get
0001:00016f00  _apr_os_sock_make
0001:00017004  _apr_os_sock_put
0001:000170b4  _apr_socket_pool_get
0001:000170c0  _apr_socket_inherit_set
0001:000170cc  _apr_socket_inherit_unset
Module: U:\extras\lib\apr-1.lib(socket_util.o)
0001:000170e0  _apr_socket_atreadeof
Module: U:\extras\lib\apr-1.lib(sockaddr.o)
0001:000171d0  _apr_sockaddr_ip_getbuf
0001:0001721c  _apr_sockaddr_ip_get
0001:00017258  _apr_sockaddr_vars_set
0001:000172a0  _apr_socket_addr_get
0001:000173c4  _apr_parse_addr_port
0001:000174d4  _apr_sockaddr_info_get
0001:000176e0  _apr_getnameinfo
0001:00017740  _apr_getservbyname
0001:000177b4  _apr_sockaddr_equal
0001:000177e4  _apr_ipsubnet_create
0001:00017a9c  _apr_ipsubnet_test
Module: U:\extras\lib\apr-1.lib(sockopt.o)
0001:00017ac0  _apr_socket_timeout_set
0001:00017ad8  _apr_socket_opt_set
0001:00017cec  _apr_socket_timeout_get
0001:00017d04  _apr_socket_opt_get
0001:00017f28  _apr_socket_atmark
0001:00017f8c  _apr_gethostname
Module: U:\extras\lib\apr-1.lib(sendrecv.o)
0001:00018000  _apr_socket_send
0001:00018144  _apr_socket_recv
0001:000182b8  _apr_socket_sendv
Module: U:\extras\lib\apr-1.lib(sendrecv_udp.o)
0001:00018430  _apr_socket_sendto
0001:0001853c  _apr_socket_recvfrom
Module: U:\extras\lib\apr-1.lib(pollset.o)
0001:00018690  _apr_pollset_create
0001:0001871c  _apr_pollset_create_ex
0001:00018728  _apr_pollset_destroy
0001:00018730  _apr_pollset_add
0001:0001878c  _apr_pollset_remove
0001:00018880  _apr_pollset_poll
Module: U:\extras\lib\apr-1.lib(poll.o)
0001:00018b60  _apr_poll
0001:00018df4  _apr_pollcb_create
0001:00018e00* _apr_pollcb_create_ex
0001:00018e0c  _apr_pollcb_add
0001:00018e18  _apr_pollcb_remove
0001:00018e24  _apr_pollcb_poll
Module: U:\extras\lib\apr-1.lib(proc_mutex.o)
0001:00018e84  _apr_proc_mutex_lockfile
0001:00018e94  _apr_proc_mutex_name
0001:00018ea0  _apr_proc_mutex_defname
0001:00018eac  _apr_proc_mutex_create
0001:00019124  _apr_proc_mutex_cleanup
0001:00018f40  _apr_proc_mutex_child_init
0001:00018fd8  _apr_proc_mutex_lock
0001:0001901c  _apr_proc_mutex_trylock
0001:00019060  _apr_proc_mutex_unlock
0001:000190a8  _apr_proc_mutex_destroy
0001:00019130  _apr_proc_mutex_pool_get
0001:0001913c  _apr_os_proc_mutex_get
0001:00019154  _apr_os_proc_mutex_put
Module: U:\extras\lib\apr-1.lib(time.o)
0001:000191a0  _apr_time_ansi_put
0001:000191d0  _apr_time_now
0001:00019204  _apr_time_exp_tz
0001:000192b0  _apr_time_exp_gmt
0001:000192dc  _apr_time_exp_lt
0001:00019308  _apr_time_exp_get
0001:00019504  _apr_time_exp_gmt_get
0001:0001953c  _apr_os_imp_time_get
0001:0001959c  _apr_os_exp_time_get
0001:000195e0  _apr_os_imp_time_put
0001:0001960c  _apr_os_exp_time_put
0001:00019650  _apr_sleep
0001:00019684  _apr_os2_time_to_apr_time
0001:00019718  _apr_apr_time_to_os2_time
0001:00019800* _apr_unix_setup_time
0001:00019870  _apr_time_clock_hires
Module: U:\extras\lib\apr-1.lib(shm.o)
0001:000198bc  _apr_shm_create
0001:0001997c  _apr_shm_destroy
0001:000199a0  _apr_shm_remove
0001:000199ac  _apr_shm_attach
0001:00019a40  _apr_shm_detach
0001:00019a68  _apr_shm_baseaddr_get
0001:00019a74  _apr_shm_size_get
0001:00019aa4  _apr_shm_pool_get
0001:00019ab0  _apr_os_shm_get
0001:00019ac4  _apr_os_shm_put
Module: U:\extras\lib\apr-1.lib(thread.o)
0001:00019b5c  _apr_threadattr_create
0001:00019ba4  _apr_threadattr_detach_set
0001:00019bb4  _apr_threadattr_detach_get
0001:00019bcc  _apr_threadattr_stacksize_set
0001:00019bdc  _apr_threadattr_guardsize_set
0001:00019be8  _apr_thread_create
0001:00019cac  _apr_os_thread_current
0001:00019cd0  _apr_thread_exit
0001:00019cec  _apr_thread_join
0001:00019d5c  _apr_thread_detach
0001:00019d70  _apr_thread_yield
0001:00019d84  _apr_os_thread_get
0001:00019d98  _apr_os_thread_put
0001:00019de4  _apr_os_thread_equal
0001:00019df8  _apr_thread_data_get
0001:00019e0c  _apr_thread_data_set
0001:00019e20  _apr_thread_pool_get
0001:00019e2c  _apr_thread_once_init
0001:00019eb8  _apr_thread_once
Module: U:\extras\lib\apr-1.lib(threadpriv.o)
0001:00019f00  _apr_threadkey_private_create
0001:00019f78  _apr_threadkey_private_get
0001:00019f8c  _apr_threadkey_private_set
0001:00019fa0  _apr_threadkey_private_delete
0001:00019fdc  _apr_threadkey_data_get
0001:00019ff0  _apr_threadkey_data_set
0001:0001a004  _apr_os_threadkey_get
0001:0001a018  _apr_os_threadkey_put
Module: U:\extras\lib\apr-1.lib(charset.o)
0001:0001a07c  _apr_os_default_encoding
0001:0001a088  _apr_os_locale_encoding
Module: U:\extras\lib\aprutil-1.lib(apr_queue.o)
0001:0001a0f4  _apr_queue_create
0001:0001a1f4  _apr_queue_push
0001:0001a2e8  _apr_queue_trypush
0001:0001a394  _apr_queue_size
0001:0001a3a0  _apr_queue_pop
0001:0001a49c  _apr_queue_trypop
0001:0001a554  _apr_queue_interrupt_all
0001:0001a59c  _apr_queue_term
Module: U:\extras\lib\apr-1.lib(sha2_glue.o)
0001:0001a62c  _apr_crypto_sha256_new
Module: U:\extras\lib\apr-1.lib(apr_random.o)
0001:0001a75c  _apr_random_init
0001:0001a894  _apr_random_after_fork
0001:0001a98c  _apr_random_standard_new
0001:0001aa20  _apr_random_add_entropy
0001:0001acb4  _apr_random_secure_bytes
0001:0001acdc  _apr_random_insecure_bytes
0001:0001ad04  _apr_random_barrier
0001:0001ad18  _apr_random_secure_ready
0001:0001ad30  _apr_random_insecure_ready
Module: U:\extras\lib\aprutil-1.lib(apr_reslist.o)
0001:0001b04c  _apr_reslist_create
0001:0001b184  _apr_reslist_destroy
0001:0001b1a8  _apr_reslist_acquire
0001:0001b390  _apr_reslist_release
0001:0001b3fc  _apr_reslist_timeout_set
0001:0001b410  _apr_reslist_acquired_count
0001:0001b440  _apr_reslist_invalidate
Module: U:\extras\lib\aprutil-1.lib(apr_rmm.o)
0001:0001b6bc  _apr_rmm_init
0001:0001b828  _apr_rmm_destroy
0001:0001b97c  _apr_rmm_attach
0001:0001b9ec  _apr_rmm_detach
0001:0001b9f4  _apr_rmm_malloc
0001:0001bb24  _apr_rmm_calloc
0001:0001bc6c  _apr_rmm_free
0001:0001be08  _apr_rmm_realloc
0001:0001bea4  _apr_rmm_addr_get
0001:0001beb4  _apr_rmm_offset_get
0001:0001bec4  _apr_rmm_overhead_get
Module: U:\extras\lib\aprutil-1.lib(sdbm.o)
0001:0001c538  _apr_sdbm_open
0001:0001c6c8  _apr_sdbm_close
0001:0001c6ec  _apr_sdbm_fetch
0001:0001c798  _apr_sdbm_delete
0001:0001c84c  _apr_sdbm_store
0001:0001c9a0  _apr_sdbm_firstkey
0001:0001ca2c  _apr_sdbm_nextkey
0001:0001ca6c  _apr_sdbm_rdonly
0001:0001ca7c  _apu__sdbm_nullitem
Module: U:\extras\lib\aprutil-1.lib(sdbm_lock.o)
0001:0001cb10  _apr_sdbm_lock
0001:0001cbf0  _apr_sdbm_unlock
Module: U:\extras\lib\aprutil-1.lib(apr_sha1.o)
0001:0001dd18  _apr_sha1_init
0001:0001dd58  _apr_sha1_update_binary
0001:0001de54  _apr_sha1_update
0001:0001de60  _apr_sha1_final
0001:0001df2c  _apr_sha1_base64
Module: U:\extras\lib\apr-1.lib(signals.o)
0001:0001dfe0  _apr_proc_kill
0001:0001e050  _apr_signal
0001:0001e0a4  _apr_signal_init
0001:0001e0c4  _apr_signal_description_get
0001:0001e0e0  _apr_signal_block
0001:0001e12c  _apr_signal_unblock
Module: U:\extras\lib\apr-1.lib(apr_strnatcmp.o)
0001:0001e398  _apr_strnatcmp
0001:0001e3ac  _apr_strnatcasecmp
Module: U:\extras\lib\apr-1.lib(apr_strings.o)
0001:0001e3c0  _apr_pstrdup
0001:0001e408  _apr_pstrndup
0001:0001e468  _apr_pstrmemdup
0001:0001e4ac  _apr_pmemdup
0001:0001e4ec  _apr_pstrcat
0001:0001e5a4  _apr_pstrcatv
0001:0001e61c  _apr_strtoff
0001:0001e67c  _apr_strtoi64
0001:0001e6b0  _apr_atoi64
0001:0001e6d4  _apr_itoa
0001:0001e74c  _apr_ltoa
0001:0001e7c0  _apr_off_t_toa
0001:0001e880  _apr_strfsize
Module: U:\extras\lib\apr-1.lib(apr_strtok.o)
0001:0001ea20  _apr_strtok
Module: U:\extras\lib\aprutil-1.lib(apr_strmatch.o)
0001:0001ebc4  _apr_strmatch_precompile
Module: U:\extras\lib\apr-1.lib(apr_tables.o)
0001:0001ee04  _apr_is_empty_array
0001:0001ee24  _apr_array_make
0001:0001ee64  _apr_array_clear
0001:0001ee74  _apr_array_pop
0001:0001eea0  _apr_array_push
0001:0001ef30  _apr_array_cat
0001:0001efe4  _apr_array_copy
0001:0001f05c  _apr_array_copy_hdr
0001:0001f09c  _apr_array_append
0001:0001f0cc  _apr_array_pstrcat
0001:0001f1c0  _apr_table_elts
0001:0001f1c8  _apr_is_empty_table
0001:0001f1e8  _apr_table_make
0001:0001f230  _apr_table_copy
0001:0001f2b8  _apr_table_clear
0001:0001f2d0  _apr_table_get
0001:0001f38c  _apr_table_set
0001:0001f5c0  _apr_table_setn
0001:0001f7b4  _apr_table_unset
0001:0001f94c  _apr_table_merge
0001:0001fab8  _apr_table_mergen
0001:0001fbf0  _apr_table_add
0001:0001fca4  _apr_table_clone
0001:0001fd00  _apr_table_addn
0001:0001fd8c  _apr_table_overlay
0001:0001fde8  _apr_table_vdo
0001:0001ff78  _apr_table_do
0001:0001ffa0  _apr_table_compress
0001:000203e0  _apr_table_overlap
Module: U:\extras\lib\apr-1.lib(thread_cond.o)
0001:000204b0  _apr_thread_cond_create
0001:000204bc  _apr_thread_cond_wait
0001:000204c8  _apr_thread_cond_timedwait
0001:000204d4  _apr_thread_cond_signal
0001:000204e0  _apr_thread_cond_broadcast
0001:000204ec  _apr_thread_cond_destroy
0001:000204f8  _apr_thread_cond_pool_get
Module: U:\extras\lib\apr-1.lib(thread_mutex.o)
0001:00020510  _apr_thread_mutex_create
0001:00020590  _apr_thread_mutex_lock
0001:000205bc  _apr_thread_mutex_trylock
0001:000205e8  _apr_thread_mutex_unlock
0001:0002060c  _apr_thread_mutex_destroy
0001:00020670  _apr_thread_mutex_pool_get
Module: U:\extras\lib\aprutil-1.lib(apr_thread_pool.o)
0001:00021260  _apr_thread_pool_create
0001:000214f4  _apr_thread_pool_destroy
0001:00021518  _apr_thread_pool_push
0001:00021544  _apr_thread_pool_schedule
0001:00021688  _apr_thread_pool_top
0001:000216f0  _apr_thread_pool_tasks_cancel
0001:000218b4  _apr_thread_pool_tasks_count
0001:000218c0  _apr_thread_pool_scheduled_tasks_count
0001:000218cc  _apr_thread_pool_threads_count
0001:000218d8  _apr_thread_pool_busy_count
0001:000218e8  _apr_thread_pool_idle_count
0001:000218f4* _apr_thread_pool_tasks_run_count
0001:00021900* _apr_thread_pool_tasks_high_count
0001:0002190c* _apr_thread_pool_threads_high_count
0001:00021918* _apr_thread_pool_threads_idle_timeout_count
0001:00021924  _apr_thread_pool_idle_max_get
0001:00021930* _apr_thread_pool_idle_wait_get
0001:00021940  _apr_thread_pool_idle_max_set
0001:00021958* _apr_thread_pool_idle_wait_set
0001:0002197c  _apr_thread_pool_thread_max_get
0001:00021988  _apr_thread_pool_thread_max_set
0001:000219fc  _apr_thread_pool_threshold_get
0001:00021a08  _apr_thread_pool_threshold_set
0001:00021a1c  _apr_thread_pool_task_owner_get
Module: U:\extras\lib\apr-1.lib(proc.o)
0001:00021b2c  _apr_procattr_create
0001:00021bb4  _apr_procattr_io_set
0001:00021ce8  _apr_procattr_child_in_set
0001:00021dc4  _apr_procattr_child_out_set
0001:00021ea0  _apr_procattr_child_err_set
0001:00021f7c  _apr_procattr_dir_set
0001:00021fa8  _apr_procattr_cmdtype_set
0001:00021fb8  _apr_procattr_detach_set
0001:00021fc8  _apr_proc_fork
0001:00022030  _apr_procattr_child_errfn_set
0001:00022038  _apr_procattr_error_check_set
0001:00022040  _apr_procattr_addrspace_set
0001:00022070  _apr_proc_create
0001:000229a0  _apr_proc_wait_all_procs
0001:00022a14  _apr_proc_wait
0001:00022b7c  _apr_proc_detach
0001:00022b88  _apr_procattr_user_set
0001:00022b94  _apr_procattr_group_set
0001:00022ba0  _apr_procattr_limit_set
Module: U:\extras\lib\apr-1.lib(otherchild.o)
0001:00022c14  _apr_proc_other_child_register
0001:00022c98  _apr_proc_other_child_unregister
0001:00022cec  _apr_proc_other_child_alert
0001:00022d5c  _apr_proc_other_child_refresh
0001:00022e08  _apr_proc_other_child_refresh_all
Module: U:\extras\lib\apr-1.lib(thread_rwlock.o)
0001:00022e40  _apr_thread_rwlock_create
0001:00022ef0  _apr_thread_rwlock_rdlock
0001:00022f48  _apr_thread_rwlock_tryrdlock
0001:00022fa0  _apr_thread_rwlock_wrlock
0001:0002300c  _apr_thread_rwlock_trywrlock
0001:00023060  _apr_thread_rwlock_unlock
0001:000230d4  _apr_thread_rwlock_destroy
0001:00023144  _apr_thread_rwlock_pool_get
Module: U:\extras\lib\apr-1.lib(timestr.o)
0001:00023150  _apr_rfc822_date
0001:00023590  _apr_day_snames
0001:00023560  _apr_month_snames
0001:00023328  _apr_ctime
0001:000234ec  _apr_strftime
Module: U:\extras\lib\aprutil-1.lib(apr_uri.o)
0001:000235b0  _apr_uri_port_of_scheme
0001:00023618  _apr_uri_unparse
0001:000238ac  _apr_uri_parse
0001:00023cb0  _apr_uri_parse_hostinfo
Module: U:\extras\lib\apr-1.lib(userinfo.o)
0001:00023f4c  _apr_uid_homepath_get
0001:00023f90  _apr_uid_current
0001:00023fb0  _apr_uid_get
0001:00023fe0  _apr_uid_name_get
Module: U:\extras\lib\apr-1.lib(groupinfo.o)
0001:00024060  _apr_gid_name_get
0001:000240d8  _apr_gid_get
Module: U:\extras\lib\aprutil-1.lib(getuuid.o)
0001:00024130  _apr_uuid_get
Module: U:\extras\lib\aprutil-1.lib(uuid.o)
0001:000243d4  _apr_uuid_format
0001:00024474  _apr_uuid_parse
Module: U:\extras\lib\apr-1.lib(version.o)
0001:00024570  _apr_version
0001:0002459c  _apr_version_string
Module: U:\extras\lib\aprutil-1.lib(xlate.o)
0001:000246e8  _apr_xlate_open
0001:00024824  _apr_xlate_sb_get
0001:0002483c  _apr_xlate_conv_buffer
0001:0002490c  _apr_xlate_conv_byte
0001:00024930  _apr_xlate_close
Module: U:\extras\lib\aprutil-1.lib(apr_xml.o)
0001:00025220  _apr_xml_parser_feed
0001:00025294  _apr_xml_parser_done
0001:00025410  _apr_xml_parser_geterror
0001:000254c4  _apr_text_append
0001:00025570  _apr_xml_quote_string
0001:0002568c  _apr_xml_quote_elem
0001:00025738  _apr_xml_to_text
0001:000257d4  _apr_xml_empty_elem
0001:0002581c  _apr_xml_insert_uri
0001:0002589c  _apr_xml_parser_create
0001:000259bc  _apr_xml_parse_file
Module: U:\extras\lib\aprutil-1.lib(apu_version.o)
0001:00025e40  _apu_version
0001:00025e6c  _apu_version_string
Module: U:\dev\httpd-2.2.20\server\.libs\main.lib(listen.o)
0001:00026144  _ap_setup_listeners
0001:000266a4  _ap_close_listeners
0001:000266e8  _ap_listen_pre_config
0001:000267fc  _ap_set_listener
0001:00026b48  _ap_set_listenbacklog
0001:00026bd0  _ap_set_send_buffer_size
0001:00026c68  _ap_set_receive_buffer_size
0002:000035b0  _ap_listeners
Module: U:\dev\httpd-2.2.20\server\mpm\mpmt_os2\.libs\mpmt_os2.lib(mpmt_os2.o)
0002:000046e0  _ap_server_conf
0001:00027324  _ap_mpm_run
0001:00027ca8  _ap_mpm_query
0001:00027d40  _ap_graceful_stop_signalled
0002:00001270  _ap_thread_stack_size
0002:00001274* _ap_max_daemons_limit
0002:00001280  _mpm_mpmt_os2_module
0002:00003604  _ap_max_spare_threads
0002:00003600  _ap_min_spare_threads
0002:00003608  _ap_my_generation
0002:0000360c  _ap_mpm_accept_mutex
Module: U:\dev\httpd-2.2.20\os\os2\.libs\os.lib(util_os2.o)
0001:000280b0  _ap_os_create_privileged_process
Module: U:\dev\httpd-2.2.20\server\.libs\main.lib(provider.o)
0001:0002810c  _ap_register_provider
0001:000282f0  _ap_lookup_provider
0001:0002835c  _ap_list_provider_names
Module: U:\dev\httpd-2.2.20\server\.libs\main.lib(util_pcre.o)
0001:00028468  _ap_regerror
0001:00028538  _ap_regfree
0001:00028550  _ap_regcomp
0001:000285cc  _ap_regexec
Module: U:\dev\httpd-2.2.20\server\.libs\main.lib(util_debug.o)
0001:00028820  _ap_strchr
0001:0002882c  _ap_strchr_c
0001:00028838  _ap_strrchr
0001:00028844  _ap_strrchr_c
0001:00028850  _ap_strstr
0001:0002885c  _ap_strstr_c
0001:00028868  _ap_get_module_config
0001:0002887c  _ap_set_module_config
Module: U:\dev\httpd-2.2.20\server\.libs\main.lib(config.o)
0001:00029470  _ap_hook_header_parser
0001:00029520  _ap_hook_get_header_parser
0001:0002952c  _ap_run_header_parser
0001:0002958c  _ap_hook_pre_config
0001:0002963c  _ap_hook_get_pre_config
0001:00029648  _ap_run_pre_config
0001:000296b8  _ap_hook_test_config
0001:00029768  _ap_hook_get_test_config
0001:00029774  _ap_run_test_config
0001:000297c8  _ap_hook_post_config
0001:00029878  _ap_hook_get_post_config
0001:00029884  _ap_run_post_config
0001:000298f4  _ap_hook_open_logs
0001:000299a4  _ap_hook_get_open_logs
0001:000299b0  _ap_run_open_logs
0001:00029a24  _ap_hook_child_init
0001:00029ad4  _ap_hook_get_child_init
0001:00029ae0  _ap_run_child_init
0001:00029b30  _ap_hook_handler
0001:00029be0  _ap_hook_get_handler
0001:00029bec  _ap_run_handler
0001:00029c4c  _ap_hook_quick_handler
0001:00029cfc  _ap_hook_get_quick_handler
0001:00029d08  _ap_run_quick_handler
0001:00029d74  _ap_hook_optional_fn_retrieve
0001:00029e24  _ap_hook_get_optional_fn_retrieve
0001:00029e30  _ap_run_optional_fn_retrieve
0001:00029e60  _ap_merge_per_dir_configs
0001:00029efc  _ap_create_request_config
0001:00029f0c  _ap_create_conn_config
0001:00029f1c  _ap_create_per_dir_config
0001:00029f98  _ap_invoke_handler
0001:0002a15c  _ap_method_is_limited
0001:0002a1cc  _ap_register_hooks
0001:0002a334  _ap_add_module
0001:0002a468  _ap_remove_module
0001:0002a518  _ap_add_loaded_module
0001:0002a55c  _ap_remove_loaded_module
0001:0002a5f4  _ap_setup_prelinked_modules
0001:0002a6d8  _ap_find_module_name
0001:0002a6e4  _ap_find_linked_module
0001:0002a720  _ap_find_command
0001:0002a768  _ap_find_command_in_modules
0001:0002abf0  _ap_set_config_vectors
0001:0002ac7c  _ap_build_cont_config
0001:0002ad84  _ap_walk_config
0001:0002af04  _ap_build_config
0001:0002b560  _ap_set_string_slot
0001:0002b5ac  _ap_set_int_slot
0001:0002b610  _ap_set_string_slot_lower
0001:0002b648  _ap_set_flag_slot
0001:0002b664  _ap_set_deprecated
0001:0002b674  _ap_server_root_relative
0001:0002b700  _ap_set_file_slot
0001:0002b77c  _ap_soak_end_container
0001:0002b958  _ap_process_resource_config
0001:0002bcd4  _ap_process_config_tree
0001:0002be68  _ap_parse_htaccess
0001:0002c0e8  _ap_init_virtual_host
0001:0002c218  _ap_fixup_virtual_hosts
0001:0002c3ac  _ap_read_config
0001:0002c788  _ap_single_module_configure
0001:0002c7e4  _ap_run_rewrite_args
0001:0002c924  _ap_show_directives
0001:0002cbcc  _ap_show_modules
0001:0002cc24  _ap_show_mpm
0002:000036b8  _ap_top_module
0002:000036bc  _ap_loaded_modules
0002:000036a4  _ap_server_root
0002:000036a8  _ap_server_pre_read_config
0002:000036ac  _ap_server_post_read_config
0002:000036a0  _ap_server_argv0
0002:000036b0  _ap_server_config_defines
0002:000036b4  _ap_conftree
Module: U:\dev\httpd-2.2.20\server\.libs\main.lib(util.o)
0001:0002cdb4  _ap_field_noparam
0001:0002ce44  _ap_ht_time
0001:0002cf60  _ap_strcmp_match
0001:0002d020  _ap_strcasecmp_match
0001:0002d108  _ap_os_is_path_absolute
0001:0002d174  _ap_is_matchexp
0001:0002d1a4  _ap_pregcomp
0001:0002d210  _ap_pregfree
0001:0002d240  _ap_strcasestr
0001:0002d340  _ap_stripprefix
0001:0002d37c  _ap_pregsub
0001:0002d52c  _ap_getparents
0001:0002d720  _ap_no2slash
0001:0002d76c  _ap_make_dirstr_prefix
0001:0002d7a4  _ap_make_dirstr_parent
0001:0002d804  _ap_count_dirs
0001:0002d830  _ap_getword
0001:0002d8c0  _ap_getword_nc
0001:0002d8d4  _ap_getword_white
0001:0002d974  _ap_getword_white_nc
0001:0002d980  _ap_getword_nulls
0001:0002d9f8  _ap_getword_nulls_nc
0001:0002da0c  _ap_getword_conf
0001:0002db48  _ap_getword_conf_nc
0001:0002db54  _ap_resolve_env
0001:0002dd30  _ap_cfg_closefile
0001:0002ddd0  _ap_pcfg_openfile
0001:0002df5c  _ap_pcfg_open_custom
0001:0002df9c  _ap_cfg_getc
0001:0002dfbc  _ap_cfg_getline
0001:0002e218  _ap_size_list_item
0001:0002e324  _ap_get_list_item
0001:0002e640  _ap_find_list_item
0001:0002eb44  _ap_get_token
0001:0002ec24  _ap_find_token
0001:0002ecbc  _ap_find_last_token
0001:0002ed3c  _ap_escape_shell_cmd
0001:0002edb0  _ap_unescape_url
0001:0002ee90  _ap_unescape_url_keep2f_ex
0001:0002ef98  _ap_unescape_url_keep2f
0001:0002efbc  _ap_construct_server
0001:0002f024  _ap_escape_path_segment
0001:0002f0ac  _ap_os_escape_path
0001:0002f190  _ap_escape_html2
0001:0002f30c  _ap_escape_html
0001:0002f330  _ap_escape_logitem
0001:0002f42c  _ap_escape_errorlog_item
0001:0002f544  _ap_is_directory
0001:0002f580  _ap_is_rdirectory
0001:0002f5bc  _ap_make_full_path
0001:0002f650  _ap_is_url
0001:0002f6a8  _ap_ind
0001:0002f6dc  _ap_rind
0001:0002f710  _ap_str_tolower
0001:0002f800  _ap_get_local_host
0001:0002f9f4  _ap_pbase64decode
0001:0002fa34  _ap_pbase64encode
0001:0002fa88  _ap_content_type_tolower
0001:0002fad0  _ap_escape_quotes
0001:0002fb78  _ap_append_pid
0001:0002fbac  _ap_timeout_parameter_parse
Module: U:\dev\httpd-2.2.20\server\.libs\main.lib(core.o)
0002:000046f0  _ap_core_input_filter_handle
0002:00004700  _ap_content_length_filter_handle
0002:00004710  _ap_core_output_filter_handle
0002:00004720  _ap_subreq_core_filter_handle
0002:00004730  _logio_add_bytes_out
0001:000328b0  _ap_core_translate
0001:00032abc  _ap_hook_get_mgmt_items
0001:00032b6c  _ap_hook_get_get_mgmt_items
0001:00032b78  _ap_run_get_mgmt_items
0001:00032bdc  _ap_add_per_dir_conf
0001:00032c04  _ap_add_per_url_conf
0001:00032c2c  _ap_add_file_conf
0001:00032c48  _ap_core_reorder_directories
0001:00032d24  _ap_allow_options
0001:00032d50  _ap_allow_overrides
0001:00032d6c  _ap_auth_type
0001:00032d88  _ap_auth_name
0001:00032db0  _ap_default_type
0001:00032dd8  _ap_document_root
0001:00032df4  _ap_requires
0001:00032e10  _ap_satisfies
0001:00032e30  _ap_response_code_string
0001:00032e84  _ap_get_remote_host
0001:000330b0  _ap_get_remote_logname
0001:000330d8  _ap_get_server_name
0001:00033178  _ap_get_server_port
0001:00033220  _ap_construct_url
0001:000332c4  _ap_get_limit_req_body
0001:000333e4  _ap_check_cmd_context
0001:000359b0  _ap_limit_section
0001:00035b4c  _ap_custom_response
0001:00035c14  _ap_exists_config_define
0001:00035d88  _ap_get_server_protocol
0001:00035da0  _ap_set_server_protocol
0001:00035e20  _ap_psignature
0001:00035fcc  _ap_get_server_revision
0001:00036004  _ap_get_server_description
0001:0003601c  _ap_get_server_banner
0001:00036034  _ap_get_server_version
0001:00036050  _ap_add_version_component
0001:00036210  _ap_get_limit_xml_body
0001:000363c8  _ap_is_recursion_limit_exceeded
0001:000364cc  _ap_add_output_filters_by_type
0001:00036554  _ap_register_request_note
0001:00036590  _ap_get_request_note
0002:000012d0  _core_module
0002:000012c0  _ap_document_root_check
Module: U:\dev\httpd-2.2.20\server\.libs\main.lib(connection.o)
0001:00037d34  _ap_hook_create_connection
0001:00037de4  _ap_hook_get_create_connection
0001:00037df0  _ap_run_create_connection
0001:00037e78  _ap_hook_process_connection
0001:00037f28  _ap_hook_get_process_connection
0001:00037f34  _ap_run_process_connection
0001:00037f94  _ap_hook_pre_connection
0001:00038044  _ap_hook_get_pre_connection
0001:00038050  _ap_run_pre_connection
0001:000380ac  _ap_flush_conn
0001:0003811c  _ap_lingering_close
0001:00038170  _ap_process_connection
Module: U:\dev\httpd-2.2.20\server\.libs\main.lib(eoc_bucket.o)
0001:000381ec  _ap_bucket_eoc_make
0001:00038270  _ap_bucket_type_eoc
0001:00038218  _ap_bucket_eoc_create
Module: U:\dev\httpd-2.2.20\server\.libs\main.lib(log.o)
0001:000382f8  _ap_logs_child_init
0001:00038324  _ap_open_stderr_log
0001:00038340  _ap_error_log2stderr
0001:00038388  _ap_close_piped_log
0001:000383b4  _ap_hook_error_log
0001:00038464  _ap_hook_get_error_log
0001:00038470  _ap_run_error_log
0001:00038a78  _ap_log_cerror
0001:00038acc  _ap_log_rerror
0001:00038b8c  _ap_log_perror
0001:00038bd8  _ap_log_error
0001:00038f54  _ap_open_piped_log_ex
0001:00039010  _ap_open_piped_log
0001:000392cc  _ap_log_assert
0001:00039364  _ap_read_pid
0001:00039538  _ap_log_pid
0001:00039c1c  _ap_open_logs
0001:00039e68  _ap_replace_stderr_log
0002:00001310  _ap_default_loglevel
Module: U:\dev\httpd-2.2.20\modules\http\.libs\mod_http.lib(http_protocol.o)
0001:0003a444  _ap_hook_insert_error_filter
0001:0003a4f4  _ap_hook_get_insert_error_filter
0001:0003a500  _ap_run_insert_error_filter
0001:0003a5c0  _ap_set_keepalive
0001:0003a984  _ap_meets_conditions
0001:0003ad34  _ap_method_registry_init
0001:0003af7c  _ap_method_register
0001:0003b050  _ap_method_number_of
0001:0003b5a4  _ap_method_name_of
0001:0003b610  _ap_index_of_response
0001:0003b648  _ap_get_status_line
0001:0003b668  _ap_send_http_options
0001:0003b6b0  _ap_set_content_type
0001:0003c76c  _ap_send_error_response
0001:0003d4d8  _ap_make_method_list
0001:0003d528  _ap_copy_method_list
0001:0003d594  _ap_method_in_list
0001:0003d628  _ap_method_list_add
0001:0003d6b8  _ap_method_list_remove
0001:0003d760  _ap_clear_method_list
Module: U:\dev\httpd-2.2.20\server\.libs\main.lib(protocol.o)
0001:0003df4c  _ap_setup_make_content_type
0001:0003dff0  _ap_make_content_type
0001:0003e11c  _ap_set_content_length
0001:0003e164  _ap_rationalize_mtime
0001:0003e1a8  _ap_rgetline_core
0001:0003e59c  _ap_getline
0001:0003e744  _ap_get_mime_headers_core
0001:0003ea54  _ap_get_mime_headers
0001:0003eb20  _ap_set_sub_req_protocol
0001:0003ed34  _ap_finalize_sub_req_protocol
0001:0003ed54  _ap_finalize_request_protocol
0001:0003edc8  _ap_note_digest_auth_failure
0001:0003ee74  _ap_note_auth_failure
0001:0003ef24  _ap_note_basic_auth_failure
0001:0003f01c  _ap_get_basic_auth_pw
0001:0003f1ec  _ap_content_length_filter
0001:0003f42c  _ap_send_fd
0001:0003f4d4  _ap_old_write_filter
0001:0003f534  _ap_rputc
0001:0003f570  _ap_rputs
0001:0003f5b8  _ap_rwrite
0001:0003f5ec  _ap_vrprintf
0001:0003f67c  _ap_rprintf
0001:0003f6b0  _ap_rvputs
0001:0003f724  _ap_rflush
0001:0003f788  _ap_set_last_modified
0001:0003f868  _ap_send_interim_response
0001:0003f9f0  _ap_hook_post_read_request
0001:0003faa0  _ap_hook_get_post_read_request
0001:0003faac  _ap_run_post_read_request
0001:0003fb10  _ap_hook_log_transaction
0001:0003fbc0  _ap_hook_get_log_transaction
0001:0003fbcc  _ap_run_log_transaction
0001:0003fc2c  _ap_hook_http_scheme
0001:0003fcdc  _ap_hook_get_http_scheme
0001:0003fce8  _ap_run_http_scheme
0001:0003fd3c  _ap_parse_uri
0001:0003fff4  _ap_read_request
0001:0004090c  _ap_hook_default_port
0001:000409bc  _ap_hook_get_default_port
0001:000409c8  _ap_run_default_port
0002:000037f0  _ap_old_write_func
Module: U:\dev\httpd-2.2.20\modules\http\.libs\mod_http.lib(http_etag.o)
0001:00040ad4  _ap_make_etag
0001:00040cd8  _ap_set_etag
Module: U:\dev\httpd-2.2.20\modules\http\.libs\mod_http.lib(http_filters.o)
0001:000416c4  _ap_http_filter
0001:000424ec  _ap_basic_http_header
0001:0004260c  _ap_http_header_filter
0001:00042e3c  _ap_discard_request_body
0001:00043008  _ap_setup_client_block
0001:00043270  _ap_should_client_block
0001:000432b8  _ap_get_client_block
0001:000434b4  _ap_send_http_trace
0001:0004378c  _ap_http_outerror_filter
Module: U:\dev\httpd-2.2.20\server\.libs\main.lib(error_bucket.o)
0001:000438a8  _ap_bucket_error_make
0001:00043980  _ap_bucket_type_error
0001:00043920  _ap_bucket_error_create
Module: U:\dev\httpd-2.2.20\modules\http\.libs\mod_http.lib(byterange_filter.o)
0001:00043b40  _ap_byterange_filter
Module: U:\dev\httpd-2.2.20\server\.libs\main.lib(request.o)
0001:00044f68  _ap_hook_translate_name
0001:00045018  _ap_hook_get_translate_name
0001:00045024  _ap_run_translate_name
0001:00045084  _ap_hook_map_to_storage
0001:00045134  _ap_hook_get_map_to_storage
0001:00045140  _ap_run_map_to_storage
0001:000451a0  _ap_hook_check_user_id
0001:00045250  _ap_hook_get_check_user_id
0001:0004525c  _ap_run_check_user_id
0001:000452b4  _ap_hook_fixups
0001:00045364  _ap_hook_get_fixups
0001:00045370  _ap_run_fixups
0001:000453d0  _ap_hook_type_checker
0001:00045480  _ap_hook_get_type_checker
0001:0004548c  _ap_run_type_checker
0001:000454ec  _ap_hook_access_checker
0001:0004559c  _ap_hook_get_access_checker
0001:000455a8  _ap_run_access_checker
0001:00045608  _ap_hook_auth_checker
0001:000456b8  _ap_hook_get_auth_checker
0001:000456c4  _ap_run_auth_checker
0001:00045724  _ap_hook_insert_filter
0001:000457d4  _ap_hook_get_insert_filter
0001:000457e0  _ap_run_insert_filter
0001:00045830  _ap_hook_create_request
0001:000458e0  _ap_hook_get_create_request
0001:000458ec  _ap_run_create_request
0001:00045cb8  _ap_directory_walk
0001:00046e10  _ap_location_walk
0001:00047120  _ap_file_walk
0001:000473d4  _ap_sub_req_output_filter
0001:00047440  _ap_some_auth_required
0001:000475b0  _ap_process_request_internal
0001:00047870  _ap_sub_req_method_uri
0001:00047974  _ap_sub_req_lookup_uri
0001:000479a0  _ap_sub_req_lookup_dirent
0001:00047cf0  _ap_sub_req_lookup_file
0001:00047f10  _ap_run_sub_req
0001:00047f6c  _ap_destroy_sub_req
0001:00047f80  _ap_update_mtime
0001:00047fa4  _ap_is_initial_req
Module: U:\dev\httpd-2.2.20\modules\http\.libs\mod_http.lib(http_request.o)
0001:00047fd0  _ap_internal_fast_redirect
0001:00048248  _ap_internal_redirect
0001:00048354  _ap_die
0001:00048a54  _ap_process_request
0001:00048be0  _ap_internal_redirect_handler
0001:00048c5c  _ap_allow_methods
0001:00048cac  _ap_allow_standard_methods
Module: U:\dev\httpd-2.2.20\server\.libs\main.lib(vhost.o)
0001:000494d4  _ap_init_vhost_config
0001:0004950c  _ap_parse_vhost_addrs
0001:00049590  _ap_set_name_virtual_host
0001:000497f0  _ap_fini_vhost_config
0001:00049ec4  _ap_matches_request_vhost
0001:00049f6c  _ap_update_vhost_from_headers
0001:0004a220  _ap_vhost_iterate_given_conn
0001:0004a2b4  _ap_update_vhost_given_ip
Module: U:\dev\httpd-2.2.20\server\.libs\main.lib(mpm_common.o)
0001:0004a58c  _ap_hook_monitor
0001:0004a63c  _ap_hook_get_monitor
0001:0004a648  _ap_run_monitor
0001:0004a69c* _ap_register_extra_mpm_process
0001:0004a6c4* _ap_unregister_extra_mpm_process
0001:0004a718* _ap_reclaim_child_processes
0001:0004a8dc* _ap_relieve_child_processes
0001:0004a9a4* _ap_mpm_safe_kill
0001:0004aa74* _ap_sock_disable_nagle
0001:0004aae8  _ap_uname2id
0001:0004ab80  _ap_gname2id
0001:0004ac30  _ap_mpm_set_pidfile
0001:0004ac78  _ap_mpm_set_max_requests
0001:0004acd0  _ap_mpm_set_max_mem_free
0002:00003c90  _ap_pid_fname
0002:00003c94  _ap_max_requests_per_child
0002:00003c98  _ap_max_mem_free
Module: U:\dev\httpd-2.2.20\server\.libs\main.lib(scoreboard.o)
0001:0004ae88* _ap_cleanup_scoreboard
0001:0004aef0  _ap_hook_pre_mpm
0001:0004afa0  _ap_hook_get_pre_mpm
0001:0004afac  _ap_run_pre_mpm
0001:0004b01c  _ap_calc_scoreboard_size
0001:0004b11c  _ap_init_scoreboard
0001:0004b21c* _ap_reopen_scoreboard
0001:0004b3b8  _ap_create_scoreboard
0001:0004b6d4  _ap_exists_scoreboard_image
0001:0004b6e8  _ap_increment_counts
0001:0004b74c* _find_child_by_pid
0001:0004b7a4  _ap_create_sb_handle
0001:0004b7d8  _ap_update_child_status_from_indexes
0001:0004ba58  _ap_update_child_status
0001:0004ba90  _ap_time_process_request
0001:0004baf0  _ap_get_scoreboard_worker
0001:0004bb34  _ap_get_scoreboard_process
0001:0004bb5c  _ap_get_scoreboard_global
0001:0004bb68  _ap_get_scoreboard_lb
0002:00003cc0  _ap_scoreboard_image
0002:00003cc4  _ap_scoreboard_fname
0002:00003cc8  _ap_extended_status
0002:00003ccc  _ap_mod_status_reqtail
Module: U:\dev\httpd-2.2.20\server\.libs\main.lib(util_filter.o)
0001:0004c268  _ap_get_output_filter_handle
0001:0004c27c  _ap_get_input_filter_handle
0001:0004c290  _ap_register_input_filter
0001:0004c2b4  _ap_register_output_filter_protocol
0001:0004c2e0  _ap_register_output_filter
0001:0004c310  _ap_add_input_filter
0001:0004c364  _ap_add_input_filter_handle
0001:0004c3c0  _ap_add_output_filter
0001:0004c414  _ap_add_output_filter_handle
0001:0004c470  _ap_remove_input_filter
0001:0004c4e0  _ap_remove_output_filter
0001:0004c550  _ap_get_brigade
0001:0004c584  _ap_pass_brigade
0001:0004c5d8  _ap_filter_flush
0001:0004c608  _ap_save_brigade
0001:0004c720  _ap_fflush
0001:0004c760  _ap_fputstrs
0001:0004c78c  _ap_fprintf
0001:0004c7bc  _ap_filter_protocol
Module: U:\dev\httpd-2.2.20\server\.libs\main.lib(util_md5.o)
0001:0004c7e4  _ap_md5_binary
0001:0004c87c  _ap_md5
0001:0004c8b0  _ap_md5contextTo64
0001:0004c978  _ap_md5digest
Module: U:\dev\httpd-2.2.20\server\.libs\main.lib(util_script.o)
0001:0004ccd0  _ap_create_environment
0001:0004cfb4  _ap_add_common_vars
0001:0004d548  _ap_find_path_info
0001:0004d658  _ap_add_cgi_vars
0001:0004da00  _ap_scan_script_header_err_core
0001:0004df34  _ap_scan_script_header_err
0001:0004df60  _ap_scan_script_header_err_brigade
0001:0004df8c  _ap_scan_script_header_err_strs
Module: U:\dev\httpd-2.2.20\server\.libs\main.lib(util_time.o)
0001:0004e178  _ap_explode_recent_localtime
0001:0004e19c  _ap_explode_recent_gmt
0001:0004e1c0  _ap_recent_ctime
0001:0004e384  _ap_recent_rfc822_date
Module: U:\dev\httpd-2.2.20\server\.libs\main.lib(util_xml.o)
0001:0004e5e4  _ap_xml_parse_input
Module: U:\tmp\ldconv_libgcc_eh_a_e34f4e5f39cd1f03c0.lib(emx-dllinit.obj)
0001:0004e8a0  _DLL_InitTerm
Module: U:\usr\lib\libend.lib(src/libend/386/endlink386.asm)
0002:000047c0  _end
0002:00003430  _edata
Module: U:\usr\lib\libend.lib(src/libend/386/end.asm)
0001:0007df50* _etext
0001:0007df50* __etext
0000:00000000* WEAK$ZERO
0002:000047c0  __end
0002:00003430  __edata
Module: U:\dev\httpd-2.2.20\modules\http\.libs\mod_http.lib(http_core.o)
0002:00004740  _ap_http_input_filter_handle
0002:00004750  _ap_http_header_filter_handle
0002:00004760  _ap_chunk_filter_handle
0002:00004770  _ap_http_outerror_filter_handle
0002:00004780  _ap_byterange_filter_handle
0002:00001390  _http_module
Module: U:\dev\httpd-2.2.20\modules\mappers\.libs\mod_so.lib(mod_so.o)
0002:000013d0  _so_module
Module: U:\tmp\ldconv_libgcc_a_e34f4e5f39ce15208.lib(__main.obj)
0001:0004fb00* ___do_global_dtors
0001:0004fb0b* ___do_global_ctors
0001:0004fb23  ___main
Module: U:\tmp\ldconv_libgcc_a_e34f4e5f39ce15208.lib(_alloca.obj)
0001:0004fb50  __alloca
Module: U:\extras\lib\aprutil-1.lib(apu_dso.o)
0001:0004fb9c  _apu_dso_mutex_lock
0001:0004fbb4  _apu_dso_mutex_unlock
0001:0004fbcc  _apu_dso_init
0001:0004fcb0  _apu_dso_load
Module: U:\extras\lib\aprutil-1.lib(apr_dbm_sdbm.o)
0001:000502d0  _apr_dbm_type_sdbm
Module: U:\usr\lib\libos2.lib(code2.obj)
0001:00050314  DosGetMessage
0001:00050300* __msgseg32
Module: U:\extras\lib\apr-1.lib(maperrorcode.o)
0001:00050364  _apr_canonical_error
Module: U:\extras\lib\apr-1.lib(filepath_util.o)
0001:00050550  _apr_filepath_list_split_impl
0001:00050610  _apr_filepath_list_merge_impl
Module: U:\extras\lib\uuid.lib(gen_uuid.obj)
0001:00050894* _uuid__generate_random
0001:00050922* _uuid_generate_random
0001:00050ea1* _uuid__generate_time
0001:000515d3* _uuid_generate_time
0001:0005177c  _uuid_generate
Module: U:\tmp\ldconv_libgcc_a_e34f4e5f39ce15208.lib(_udivdi3.obj)
0001:000517e0  ___udivdi3
Module: U:\extras\lib\apr-1.lib(os2calls.o)
0002:00004790  _apr_os2_sendto
0002:000047a0  _apr_os2_recvfrom
0002:000015d0  _apr_os2_socket
0002:00004550  _apr_os2_select
0002:00004554  _apr_os2_sock_errno
0002:00004558  _apr_os2_accept
0002:0000455c  _apr_os2_bind
0002:00004560  _apr_os2_connect
0002:00004564  _apr_os2_getpeername
0002:00004568  _apr_os2_getsockname
0002:0000456c  _apr_os2_getsockopt
0002:00004570  _apr_os2_ioctl
0002:00004574  _apr_os2_listen
0002:00004578  _apr_os2_recv
0002:0000457c  _apr_os2_send
0002:00004580  _apr_os2_setsockopt
0002:00004584  _apr_os2_shutdown
0002:00004588  _apr_os2_soclose
0002:0000458c  _apr_os2_writev
Module: U:\extras\lib\apr-1.lib(inet_ntop.o)
0001:00051d60  _apr_inet_ntop
Module: U:\extras\lib\apr-1.lib(inet_pton.o)
0001:00051e60  _apr_inet_pton
Module: U:\tmp\ldconv_libgcc_a_e34f4e5f39ce15208.lib(_divdi3.obj)
0001:00051f50  ___divdi3
Module: U:\extras\lib\apr-1.lib(waitio.o)
0001:000520a0  _apr_wait_for_io_or_timeout
Module: U:\tmp\ldconv_libgcc_a_e34f4e5f39ce15208.lib(_moddi3.obj)
0001:000521b0  ___moddi3
Module: U:\extras\lib\apr-1.lib(sha2.o)
0001:00052370  _apr__SHA256_Init
0001:000523a8* _apr__SHA256_Transform
0001:00052624  _apr__SHA256_Update
0001:00052764  _apr__SHA256_Final
0001:000528b8* _apr__SHA256_End
0001:0005294c* _apr__SHA256_Data
0001:00052990* _apr__SHA512_Init
0001:000529d8* _apr__SHA512_Transform
0001:000530d0* _apr__SHA512_Update
0001:0005329c* _apr__SHA512_Last
0001:000533b8* _apr__SHA512_Final
0001:00053438* _apr__SHA512_End
0001:000534cc* _apr__SHA512_Data
0001:00053514* _apr__SHA384_Init
0001:0005355c* _apr__SHA384_Update
0001:00053584* _apr__SHA384_Final
0001:00053604* _apr__SHA384_End
0001:00053698* _apr__SHA384_Data
Module: U:\extras\lib\aprutil-1.lib(sdbm_pair.o)
0001:00053b70  _apu__sdbm_fitpair
0001:00053ba4  _apu__sdbm_putpair
0001:00053c10  _apu__sdbm_getpair
0001:00053c58  _apu__sdbm_duppair
0001:00053c90  _apu__sdbm_getnkey
0001:00053cdc  _apu__sdbm_delpair
0001:00053db4  _apu__sdbm_splpage
0001:00053ea0  _apu__sdbm_chkpage
Module: U:\extras\lib\aprutil-1.lib(sdbm_hash.o)
0001:00053f10  _apu__sdbm_hash
Module: U:\extras\lib\expat.lib(xmlparse.obj)
0001:00054073* _XML_UseParserAsHandlerArg
0001:0005407e* _XML_UseForeignDTD
0001:000540a8* _XML_SetReturnNSTriplet
0001:000540cc  _XML_SetUserData
0001:000540e7* _XML_GetBase
0001:000540f5* _XML_GetSpecifiedAttributeCount
0001:00054103* _XML_GetIdAttributeIndex
0001:00054111  _XML_SetElementHandler
0001:00054125* _XML_SetStartElementHandler
0001:00054133* _XML_SetEndElementHandler
0001:00054141  _XML_SetCharacterDataHandler
0001:0005414f* _XML_SetProcessingInstructionHandler
0001:0005415d* _XML_SetCommentHandler
0001:0005416b* _XML_SetCdataSectionHandler
0001:0005417f* _XML_SetStartCdataSectionHandler
0001:0005418d* _XML_SetEndCdataSectionHandler
0001:0005419b  _XML_SetDefaultHandler
0001:000541b0* _XML_SetDefaultHandlerExpand
0001:000541c5* _XML_SetDoctypeDeclHandler
0001:000541d9* _XML_SetStartDoctypeDeclHandler
0001:000541e7* _XML_SetEndDoctypeDeclHandler
0001:000541f5* _XML_SetUnparsedEntityDeclHandler
0001:00054203* _XML_SetNotationDeclHandler
0001:00054211* _XML_SetNamespaceDeclHandler
0001:00054225* _XML_SetStartNamespaceDeclHandler
0001:00054233* _XML_SetEndNamespaceDeclHandler
0001:00054241* _XML_SetNotStandaloneHandler
0001:0005424f* _XML_SetExternalEntityRefHandler
0001:0005425d* _XML_SetExternalEntityRefHandlerArg
0001:00054274* _XML_SetSkippedEntityHandler
0001:00054282* _XML_SetUnknownEncodingHandler
0001:00054299* _XML_SetElementDeclHandler
0001:000542aa* _XML_SetAttlistDeclHandler
0001:000542bb* _XML_SetEntityDeclHandler
0001:000542cc* _XML_SetXmlDeclHandler
0001:000542dd* _XML_SetParamEntityParsing
0001:00054307* _XML_ParseBuffer
0001:00054438* _XML_StopParser
0001:000544af* _XML_ResumeParser
0001:00054598  _XML_GetErrorCode
0001:000545a6* _XML_GetCurrentByteIndex
0001:000545c5* _XML_GetCurrentByteCount
0001:000545e7* _XML_GetInputContext
0001:00054618* _XML_GetCurrentLineNumber
0001:00054671* _XML_GetCurrentColumnNumber
0001:000546c7* _XML_FreeContentModel
0001:000546dc* _XML_MemMalloc
0001:000546f1* _XML_MemRealloc
0001:0005470c* _XML_MemFree
0001:00054721  _XML_ErrorString
0001:00054746* _XML_ExpatVersion
0001:00054750* _XML_ExpatVersionInfo
0001:0005476e* _XML_GetFeatureList
0001:00054866* _XML_DefaultCurrent
0001:00055029  _XML_ParserFree
0001:0005547a* _XML_GetParsingStatus
0001:000554c0* _XML_GetBuffer
0001:00055642  _XML_Parse
0001:00055995* _XML_SetBase
0001:000559df* _XML_SetEncoding
0001:0005744a* _XML_ExternalEntityParserCreate
0001:00057a6d* _XML_ParserReset
0001:00057dc1* _XML_ParserCreate_MM
0001:00057e0e* _XML_ParserCreateNS
0001:00057e36  _XML_ParserCreate
Module: U:\dev\httpd-2.2.20\server\mpm\mpmt_os2\.libs\mpmt_os2.lib(mpmt_os2_child.o)
0002:000047b0+ _shutdown_event
0001:0005d724* thread_exception_handler
0001:0005dcd0  _ap_mpm_child_main
0001:0005e4a4* _add_worker
Module: U:\dev\httpd-2.2.20\srclib\pcre\.libs\pcre.lib(pcre.o)
0001:000649b4* _pcre_version
0001:000649c0  _pcre_info
0001:00064a44* _pcre_fullinfo
0001:00064bc4* _pcre_config
0001:00064ecc  _pcre_compile
0001:00066514  _pcre_exec
0002:00002364  _pcre_free
0002:00002360* _pcre_malloc
0002:00002368* _pcre_stack_malloc
0002:0000236c* _pcre_stack_free
0002:000045d0* _pcre_callout
Module: U:\dev\httpd-2.2.20\server\.libs\main.lib(util_cfgtree.o)
0001:000670c0  _ap_add_node
Module: U:\dev\httpd-2.2.20\server\.libs\main.lib(core_filters.o)
0001:00067400  _ap_core_input_filter
0001:0006798c  _ap_core_output_filter
Module: U:\usr\lib\tcpipv4\libc_dll.lib(syslog.obj)
0001:0006859c  _syslog
0001:00068604* _vsyslog
0001:00068a5c  _openlog
0001:00068aac* _closelog
0001:00068ae0* _setlogmask
Module: U:\tmp\ldconv_libgcc_a_e34f4e5f39ce15208.lib(emx-ctordtor.obj)
0001:00068b10  ___ctordtorInit
0001:00068b42  ___ctordtorTerm
Module: U:\tmp\ldconv_libgcc_eh_a_e34f4e5f39cd1f03c0.lib(emx-eh.obj)
0001:00068b80  ___ehInit
0001:00068bb5* ___ehTerm
Module: U:\dev\httpd-2.2.20\modules\http\.libs\mod_http.lib(chunk_filter.o)
0001:00068c00  _ap_http_chunk_filter
Module: U:\extras\lib\uuid.lib(unpack.obj)
0001:00068f10  _uuid_unpack
Module: U:\extras\lib\uuid.lib(pack.obj)
0001:00068f80  _uuid_pack
Module: U:\usr\lib\tcpipv4\libc_dll.lib(socket.obj)
0001:00068fe0  _socket
Module: U:\usr\lib\tcpipv4\libc_dll.lib(connect.obj)
0001:00069060  _connect
Module: U:\tmp\ldconv_libgcc_eh_a_e34f4e5f39cd1f03c0.lib(emutls.obj)
0001:000691b3  ___emutls_get_address
0001:0006949f* ___emutls_register_common
Module: U:\extras\lib\expat.lib(xmlrole.obj)
0001:0006ae50  _XmlPrologStateInit
0001:0006ae73  _XmlPrologStateInitExternalEntity
Module: U:\extras\lib\expat.lib(xmltok.obj)
0001:00079e6f  _XmlUtf8Encode
0001:00079f0f* _XmlUtf16Encode
0001:00079f57  _XmlSizeOfUnknownEncoding
0001:0007a18c  _XmlInitUnknownEncoding
0001:0007a6b2  _XmlGetUtf8InternalEncoding
0001:0007a6bc* _XmlGetUtf16InternalEncoding
0001:0007a723  _XmlInitEncoding
0001:0007a815  _XmlParseXmlDecl
0001:0007a865  _XmlGetUtf8InternalEncodingNS
0001:0007a86f* _XmlGetUtf16InternalEncodingNS
0001:0007a8d6  _XmlInitEncodingNS
0001:0007a9c8  _XmlParseXmlDeclNS
0001:0007aa18  _XmlInitUnknownEncodingNS
Module: U:\tmp\ldconv_libgcc_eh_a_e34f4e5f39cd1f03c0.lib(unwind-dw2-fde.obj)
0001:0007d891* ___register_frame_info_bases
0001:0007d990* ___register_frame_info
0001:0007d9bb* ___register_frame
0001:0007d9e6* ___register_frame_info_table_bases
0001:0007dad8* ___register_frame_info_table
0001:0007db03  ___register_frame_table
0001:0007db26* ___deregister_frame_info_bases
0001:0007dc8e* ___deregister_frame_info
0001:0007dc99  ___deregister_frame
0001:0007dcbe* __Unwind_Find_FDE
Module: U:\usr\lib\tcpipv4\libc_dll.lib(send.obj)
0001:0007dea0* _send


                        +----------------------+
                        |   Imported Symbols   |
                        +----------------------+

Symbol                              Module
======                              ======

___libc_ForkRegisterModule          libc063
___init_dll                         libc063
___libc_Back_termDll                libc063
___libc_ForkDeregisterModule        libc063
__atfork_callback                   libc063
___stderrp                          libc063
___libc_GLocaleCtype                libc063
DosFreeModule                       doscalls
DosLoadModule                       doscalls
DosQueryModuleHandle                doscalls
DosQueryProcAddr                    doscalls
__errno                             libc063
DosQueryFileInfo                    doscalls
DosQueryPathInfo                    doscalls
DosQueryHType                       doscalls
DosFindFirst                        doscalls
DosSetPathInfo                      doscalls
DosFindClose                        doscalls
DosFindNext                         doscalls
DosCreateDir                        doscalls
DosDeleteDir                        doscalls
DosQueryCurrentDir                  doscalls
DosQueryCurrentDisk                 doscalls
DosSetCurrentDir                    doscalls
DosSetDefaultDisk                   doscalls
DosOpen                             doscalls
DosSetFilePtr                       doscalls
DosClose                            doscalls
DosSetRelMaxFH                      doscalls
DosDelete                           doscalls
DosMove                             doscalls
DosQueryFHState                     doscalls
DosSetFHState                       doscalls
DosWrite                            doscalls
DosSetFileLocks                     doscalls
DosRead                             doscalls
DosResetEventSem                    doscalls
DosWaitEventSem                     doscalls
DosDupHandle                        doscalls
DosSetFileSize                      doscalls
DosCreateNPipe                      doscalls
DosConnectNPipe                     doscalls
DosCreateEventSem                   doscalls
DosSetNPipeSem                      doscalls
DosCloseEventSem                    doscalls
DosSetNPHState                      doscalls
__assert                            libc063
___stdoutp                          libc063
gethostbyname                       tcp32dll
inet_addr                           tcp32dll
tcp_h_errno                         tcp32dll
gethostbyaddr                       tcp32dll
getservbyname                       tcp32dll
gethostname                         tcp32dll
DosCreateMutexSem                   doscalls
DosOpenMutexSem                     doscalls
DosRequestMutexSem                  doscalls
___threadid                         libc063
DosReleaseMutexSem                  doscalls
DosCloseMutexSem                    doscalls
DosSleep                            doscalls
DosAllocSharedMem                   doscalls
DosFreeMem                          doscalls
DosGetNamedSharedMem                doscalls
DosGetSharedMem                     doscalls
DosQueryMem                         doscalls
__beginthread                       libc063
DosGetInfoBlocks                    doscalls
__endthread                         libc063
DosWaitThread                       doscalls
DosAllocThreadLocalMemory           doscalls
DosFreeThreadLocalMemory            doscalls
DosSendSignalException              doscalls
_sys_siglist                        libc063
DosEnterCritSec                     doscalls
__getcwd2                           libc063
__chdir2                            libc063
DosExecPgm                          doscalls
DosExitCritSec                      doscalls
DosSearchPath                       doscalls
DosWaitChild                        doscalls
DosPostEventSem                     doscalls
_getpwnam_r                         libc063
_getpwuid_r                         libc063
_getgrgid_r                         libc063
_getgrnam_r                         libc063
DosQueryModuleName                  doscalls
_getpwnam                           libc063
__CRT_init                          libc063
__std_exit                          libc063
__std_fprintf                       libc063
__std_printf                        libc063
__std_puts                          libc063
__std_stricmp                       libc063
__std_strnicmp                      libc063
__std_malloc                        libc063
__std_free                          libc063
__std_memchr                        libc063
__std_strchr                        libc063
__std_atoi                          libc063
__std_sprintf                       libc063
__std_strcat                        libc063
__std_getenv                        libc063
__std_setenv                        libc063
__std_unsetenv                      libc063
DosTrueGetMessage                   msg
__std_strerror                      libc063
__std_strerror_r                    libc063
__std_fstat                         libc063
__std_access                        libc063
__std_strncmp                       libc063
__std_memcmp                        libc063
__std_close                         libc063
__std_unlink                        libc063
__std_write                         libc063
__std_lseek                         libc063
__std_writev                        libc063
__std_getpid                        libc063
__std_mkstemp                       libc063
__std_setmode                       libc063
__std_fcntl                         libc063
__std_strrchr                       libc063
__std_random                        libc063
__std_qsort                         libc063
__std_strcmp                        libc063
__std_fputc                         libc063
__std_fwrite                        libc063
__std_fputs                         libc063
__std_modf                          libc063
__std_getpass                       libc063
__std_strncat                       libc063
__std_strspn                        libc063
__std_strtol                        libc063
__std_strcpy                        libc063
__std_gettimeofday                  libc063
__std_gmtime_r                      libc063
__std_timezone                      libc063
__std_mktime                        libc063
__std_localtime                     libc063
__std_difftime                      libc063
__std_nl_langinfo                   libc063
__std_kill                          libc063
__std_sigemptyset                   libc063
__std_sigaction                     libc063
__std_sigaddset                     libc063
__std_sigprocmask                   libc063
__std_strtoll                       libc063
__std_fork                          libc063
__std_strpbrk                       libc063
__std_chdir                         libc063
__std_waitpid                       libc063
__std_strftime                      libc063
__std_getuid                        libc063
__std_getgid                        libc063
__std_srand                         libc063
__std_rand                          libc063
__std_iconv_close                   libc063
__std_iconv                         libc063
__std_iconv_open                    libc063
__std_signal                        libc063
__std_getppid                       libc063
__gettid                            libc063
DosUnwindException                  doscalls
DosSetExceptionHandler              doscalls
DosOpenQueue                        quecalls
DosReadQueue                        quecalls
DosSetSignalExceptionFocus          doscalls
DosCreateQueue                      quecalls
DosWriteQueue                       quecalls
DosPurgeQueue                       quecalls
DosKillThread                       doscalls
DosQueryQueue                       quecalls
__std_remove                        libc063
__std_strncpy                       libc063
__std_strstr                        libc063
__std_putchar                       libc063
__std_atol                          libc063
__std_time                          libc063
__std_ctime_r                       libc063
__getprogname                       libc063
__std_vsnprintf                     libc063
__std_open                          libc063
__std_memset                        libc063
__std_abort                         libc063
__std_freopen                       libc063
__std_sscanf                        libc063
__std_getpgid                       libc063
__std_getpgrp                       libc063
__std_getgrnam                      libc063
__std_calloc                        libc063
__std_times                         libc063
___ctordtorInit1                    libc063
___ctordtorTerm1                    libc063
__std_atexit                        libc063
__std_srandom                       libc063
__std_read                          libc063
__libsocket_socket                  so32dll
___libc_TcpipAllocFH43              libc063
__libsocket_soclose                 so32dll
__libsocket_set_errno               so32dll
__libsocket_sock_errno              so32dll
___libc_FH                          libc063
__libsocket_connect                 so32dll
___libc_TLSSet                      libc063
__fmutex_create                     libc063
___libc_TLSAlloc                    libc063
___libc_TLSDestructor               libc063
___libc_TLSGet                      libc063
___libc_Back_threadSleep            libc063
___libc_GpFIBLIS                    libc063
___fmutex_release_internal          libc063
___fmutex_request_internal          libc063
___fmutex_release_internal_must_complete libc063
___fmutex_request_internal_must_complete libc063
__std_stat                          libc063
__std_sysconf                       libc063
__std_execl                         libc063
__std_ioctl                         libc063
__std_rewind                        libc063
__std_fclose                        libc063
__std_fflush                        libc063
__std_ftruncate                     libc063
__std_umask                         libc063
__std_fdopen                        libc063
__std_fscanf                        libc063
__std_memmove                       libc063
__std_memcpy                        libc063
__std_realloc                       libc063
__libsocket_send                    so32dll


                        +--------------------+
                        |   Libraries Used   |
                        +--------------------+

U:\dev\httpd-2.2.20\server\.libs\main.lib
U:\dev\httpd-2.2.20\modules\http\.libs\mod_http.lib
U:\dev\httpd-2.2.20\modules\mappers\.libs\mod_so.lib
U:\dev\httpd-2.2.20\server\mpm\mpmt_os2\.libs\mpmt_os2.lib
U:\dev\httpd-2.2.20\os\os2\.libs\os.lib
U:\dev\httpd-2.2.20\srclib\pcre\.libs\pcre.lib
U:\extras\lib\aprutil-1.lib
U:\extras\lib\expat.lib
U:\extras\lib\apr-1.lib
U:\extras\lib\uuid.lib
U:\tmp\ldconv_libgcc_eh_a_e34f4e5f39cd1f03c0.lib
U:\tmp\ldconv_libgcc_a_e34f4e5f39ce15208.lib
U:\usr\lib\libc_alias.lib
U:\usr\lib\tcpipv4\libc_dll.lib
U:\usr\lib\libos2.lib
U:\usr\lib\libend.lib


                        +-----------------------+
                        |   Linker Statistics   |
                        +-----------------------+

Stack size:  0000 (0.)
Memory size:  00082710 (534288.)
Link time: 00:00.12
